S31508001800A80A0020D9180008E7180008E9180008EF
S3150800181000000000000000000000000000000000BA
S315080018200000000000000000000000000119000888
S31508001830000000000000000003190008893C0008A9
S31508001840654E000807190008071900080719000857
S3150800185007190008071900080719000807190008DA
S3150800186007190008052A00080719000807190008BB
S3150800187007190008071900080719000807190008BA
S3150800188007190008000000000000000007190008FA
S3150800189000000000071900080719000807190008C2
S315080018A00000000007190008071900084D4700083E
S315080018B007190008071900080719000800000000A2
S315080018C0EE11AA550348854600F03AFD0048004740
S315080018D0A9830008A80A00200B4880F308880B484B
S315080018E080470B480047FEE704207146084202D0AD
S315080018F0EFF3098001E0EFF30880714606F0A0FBDC
S31508001900FEE7FEE7FEE7FEE7A80A0020253F0008F7
S31508001910C518000830B50B460146002020220124D0
S3150800192009E00D46D5409D4205D31D469540491B05
S315080019302546954040191546521E002DF1DC30BD4E
S3150800194070B500242546002801DA01244042002902
S3150800195001DA01254942FFF7DDFFAC4200D04042DB
S31508001960002C00D0494270BD03460B439B0703D0A9
S3150800197009E008C9121F08C0042AFAD203E00B7846
S315080019800370401C491C521EF9D27047D2B201E0BE
S315080019900270401C491EFBD270470022F6E710B5BC
S315080019A013460A4604461946FFF7F0FF204610BDBF
S315080019B0F8B502464A40D40F42004B0052085B086D
S315080019C09A4202D20246084611464A0023D0C30D5F
S315080019D04A00DDB2120EAD1A202D35DA490201266B
S315080019E0490AF6058A19002C00D0524220214F1BBD
S315080019F01146B9402A411018C20D9A4221D0002C2E
S31508001A0017D0012D08DCDA05801AD20F8019D20703
S31508001A10DBB200F077FBF8BDDA05801A0123400037
S31508001A201B06C01880185A428018CA0F104349006E
S31508001A3007E04908C2071143DA05801A80194008E9
S31508001A40801800F057FBF8BD61000122511A001BEF
S31508001A50F7E70122D2075140AAE70122D2075040F0
S31508001A60A6E7024670B54A40D30FDB0740002DD0E3
S31508001A704A002AD0010E140E000212020919400A61
S31508001A80520A8418E50104465443000A120A2E0431
S31508001A905043A4194219200CC543AA18120C012553
S31508001AA0AD03521C521912047F39240400D0521C6B
S31508001AB0104301D44000491EC2B20C06C0092018C2
S31508001AC0401C4008802A02D003E0002070BD400870
S31508001AD04000002900DA0020184370BD70B50246A0
S31508001AE04A40D50F40004A00ED0740085208002832
S31508001AF014D0002A12D0C40DD30D41020120C0050E
S31508001B005202490A520AE41A091812187D349142F7
S31508001B1001D3641C00E04900002C01DA002070BDE6
S31508001B200023914201D3891A03434008490000283B
S31508001B30F7D100290AD0914202D10121C90705E04F
S31508001B40914201D2012101E00121C943E005C018F3
S31508001B50401900F0CFFA70BDF0B507460846584060
S31508001B6087B0C00F049048000E465900400849083F
S31508001B70BC1A884105D2384631461E4617460B46DA
S31508001B8002465800400810434CD0300D03904005DB
S31508001B905900400D490D0590401A0290402872DA06
S31508001BA018030121000B09050843019004980092C7
S31508001BB0002805D0019952420020884100920190E0
S31508001BC0029840210A1A0199009800F05FFA054622
S31508001BD00C466B4607CB00F07AFAC0197141039A96
S31508001BE00E0D0023D71756401A467A40164344D09E
S31508001BF0049A002A2DD0029A012A039A15DC1205A6
S31508001C00C01A914101263605001C7141D20F059E66
S31508001C10D2070093019202962A46234600F0B8FAA4
S31508001C2007B0F0BD38463146FAE71605224A0F4690
S31508001C30B218C01AB74101210905001C4F41001806
S31508001C407F41114618187941E20F10436D19644116
S31508001C5013E0E2076D0815436408C2071443039AA4
S31508001C6001261205C01A91413605001C7141CE079E
S31508001C70400830434908C01851412A46234600F017
S31508001C807AFACDE7FFE7049801224000C117121A35
S31508001C9000238B4104983146C417381AA141EEE750
S31508001CA030B40124E407634030BC55E730B401245E
S31508001CB0E407614030BC4FE70000E0FFF0B51FB411
S31508001CC088B00B990998002448400999C00F490023
S31508001CD049080991C0070B990090490049080B91DA
S31508001CE009990898A64608431CD00B990A980843F0
S31508001CF018D0099801244000420D4800410D099862
S31508001D0024050003000B204309900B980003000BE1
S31508001D1020430B9050181C49401800220190144685
S31508001D20104605E0002001460DB0F0BD032801DA93
S31508001D30034600E003239C46C11A0AAE0AE05F0088
S31508001D4008ADED5B4F00F75B7D430027AA187C4181
S31508001D50491C5B1E6145F2DD410004AB5A52210461
S31508001D60120C0A43240C401C0828DFDB0198029059
S31508001D700099704601910090059B049A0799069868
S31508001D8000F006FAD0E700000DFCFFFFF0B50C46A0
S31508001D905C4085B0E40FE40703944C000026640811
S31508001DA059009446490802460296224321D06246C3
S31508001DB00A431ED06200570D4A000E032303550D31
S31508001DC0012402462C492405781B1B0B360B4018A8
S31508001DD023432643614600901C46501AB44103D358
S31508001DE00098401C009002E0921800985B41002879
S31508001DF003DA0020014605B0F0BD002001210905DF
S31508001E000746864611E064461D46141BB54106D3AF
S31508001E106546521BB341744607430C43A646CD0795
S31508001E2040084908284392185B4105460D43EAD104
S31508001E301046184313D0604619465040714008436F
S31508001E4006D06046101AB34106D20122002306E0E6
S31508001E5000220123DB0702E00122D2435310009837
S31508001E6074460105381C6141029C039D00196941AD
S31508001E7000F081F9BFE70000FD030000C217C10F9B
S31508001E80504010B54018CA079623002100F03AF9C9
S31508001E9010BD10B500229623114600F033F910BD87
S31508001EA00EB5C217C10F5040CA0740180021054B8E
S31508001EB00293019200910A460B4600F069F903B0B5
S31508001EC000BD0000330400000EB50549029100214B
S31508001ED000910A460B46019100F05AF903B000BD7D
S31508001EE033040000C20F410040020123400ADB050B
S31508001EF0D207090EC0187F2901DA002070479629F3
S31508001F0003DC9623591AC84001E096398840002A0E
S31508001F10F4D040427047410040020122400AD205EF
S31508001F20090E80187F2901DA00207047962903DCFC
S31508001F309622511AC8407047963988407047000063
S31508001F404A0009030123090B1B051943094B10B560
S31508001F50520D9A4201DA002010BD064B34339A42DC
S31508001F6003DC9A1A00F0A2F810BD034951188840FC
S31508001F7010BD0000FF030000CDFBFFFFC20FD20714
S31508001F80400040080BD0C10D0723DB01C9184002E9
S31508001F900905400A1143C20840071143704700204B
S31508001FA00146704710B5002904DB0124E4074042C6
S31508001FB08C412146002B04DB1C460123DB075242D9
S31508001FC0A3418B4200D1824210BD0000CB0FDB0734
S31508001FD0490010B5490802460A4307D00A0D0724E6
S31508001FE00903E401090B121B002A01DC002010BDBD
S31508001FF0C900440F0C43C100E018D205801800F050
S3150800200079F810BD0122D207002800DB101A002932
S3150800201000DB511A814270470122D207002800DBF3
S31508002020101A002900DB511A88427047F0B51FB410
S315080020300646002082B005464024019100901BE028
S31508002040019922460F46304600F030F8049A059B5F
S31508002050801A994110D310461946224600F016F800
S31508002060361A8F410197224601200021009F00F071
S315080020700DF838184D4100902046641E0028DFDC14
S31508002080019B00982946324607B0F0BD10B5202AB4
S3150800209004DB0146203A9140002010BD91402023E0
S315080020A09C1A0346E3401943904010BD10B5202AF8
S315080020B004DB0846203AD040002110BD0B46D34029
S315080020C0D0402024A21A91400843194610BD10B5E5
S315080020D0202A06DBCB170846203A1041C1170B43C6
S315080020E006E00B461341D0402024A21A914008432B
S315080020F0194610BD002904DA401C490001D14008E0
S315080021004000704770B40024050C05D11024000463
S3150800211002D1002921D01124050E01D1000208346C
S31508002120050F01D10001241D850F01D18000A41CD3
S31508002130002801DB4000641C002908D020252E1B3E
S315080021400D46F540A14000D0012129430843010668
S315080021501B1B000ADB1D02D5002070BC7047DB057F
S31508002160181880180029F8DA401C4900F5D170BC07
S3150800217040084000704710B5002B08DA0024401CC0
S31508002180614192185B411A4301D14008400010BDD5
S31508002190F0B51FB482B005460C0003D0084602F01D
S315080021A0E7FE02E002F0E4FE2030024600902146F7
S315080021B02846FFF76BFF049B059A04460F4618430B
S315080021C01143084314D0184610431BD000984021E9
S315080021D00A1A18460599FFF769FF05460E46009A3A
S315080021E005990498FFF752FF084305D0012004E03B
S315080021F02046394607B0F0BD0020C11705430E43F7
S315080022002C43374300990E986305401A7905E40A6A
S3150800221000220C43FD0A0A3002D500200146E9E7F0
S315080022200105101969410C9C0D9D00196941FFF7BC
S31508002230A2FFDFE7FEB500231A461B1A8A4103DB15
S315080022400020014603B0F0BD4A000D0301212D0B05
S315080022500905520D0D43D10702D100186D41521ED2
S315080022605110FF31FF310131002704463E463846FA
S31508002270009701910246012100200905FFF716FF84
S31508002280C3197141F818324684468E464A4161465A
S315080022902846611A904104D36046241A9541764629
S315080022A01F46241900986D41401C00903428E1DD32
S315080022B0F91930467041091BA84103D20022D243BE
S315080022C0134601E00022134601980105381C7141A6
S315080022D0FFF751FFB6E700004A0009030123090B7F
S315080022E01B0519430A4B10B5520D9A4202DA002013
S315080022F0014610BD064B34339A4203DC9A1AFFF79F
S31508002300D5FE10BD034BD218FFF7C0FE10BD000066
S31508002310FF030000CDFBFFFF10B5002904DB0124F5
S31508002320E40740428C412146002B04DB1C4601236E
S31508002330DB075242A341994200D1904210BD0000EA
S31508002340064C0125064E05E0E36807CC2B430C3CFA
S3150800235098471034B442F7D3FFF7B8FAC0A4000878
S31508002360E0A4000870B58C180578401C6B075B0F55
S3150800237001D10378401C2A1106D10278401C03E0DB
S3150800238006780E70401C491C5B1EF9D12B0705D434
S315080023900023521E0DD40B70491CFAE70378401C23
S315080023A0CB1A921C03E01D780D70491C5B1C521E4B
S315080023B0F9D5A142D8D3002070BD000010B5044657
S315080023C0002C08D101210920C00600F0E7FD0020F5
S315080023D000F0E6F852E0012C05D102210920C006DA
S315080023E000F0DCFD4AE0022C05D104210920C006D4
S315080023F000F0D4FD42E0032C05D108210920C006CF
S3150800240000F0CCFD3AE0042C05D110210920C006C5
S3150800241000F0C4FD32E0052C05D120210920C006B4
S3150800242000F0BCFD2AE0062C05D140210920C00693
S3150800243000F0B4FD22E0072C05D180210920C00652
S3150800244000F0ACFD1AE0082C04D101210D4800F07B
S31508002450A5FD13E0092C04D102210A4800F09EFDCF
S315080024600CE00B2C04D11021064800F097FD05E07E
S315080024700C2C03D18021034800F090FD204600F083
S315080024808FF810BD000400487FB500200090019029
S3150800249002900390002427E000250CE0E800294973
S315080024A040186100405AA1006A4651584018A100D8
S315080024B05050681C85B2142DF0DBA1006A465058AE
S315080024C01421FFF727FA2821484361001E4A515A6A
S315080024D03C225143461864213046FFF71BFA610037
S315080024E0194A5052601C84B2042CD5DB1748C07CAC
S315080024F0002826D0144840881549884203DC12482B
S31508002500808888420ADD11482038C078002805D11D
S315080025101049486005210D482038C1700A4840888E
S315080025200A2803DB084880880A280ADA0748203878
S31508002530C078002805D10749486004210348203897
S31508002540C1707FBDEC040020740100202C0400201B
S31508002550E60F00000C02002000B587B001A800F0C5
S31508002560AFF80121480201F001FA0020019070201D
S31508002570029001208002039000200690059001A990
S31508002580064800F031F80121044800F021F801213D
S31508002590024800F011F807B000BD00000024014011
S315080025A010B50446072300222146024800F038F8F1
S315080025B010BD000000240140002904D04268012310
S315080025C01A43426003E0426852085200426070476C
S315080025D0002904D0826808231A43826003E08268CF
S315080025E008239A438260704742680B4B1A40426040
S315080025F00B684A681A4343681A4342608268074B65
S315080026001A4082600B694A691A438B681A438368C1
S315080026101A438260704700000FBCFFFF8FF1F9FF75
S31508002620F0B504460D4616461F463F073F0F2B4694
S31508002630082B0FD91B071B0F083B606F9A000F2149
S31508002640914088436067606F99003A468A40104314
S3150800265060670BE0206F9A000F219140884320673E
S31508002660206F99003A468A4010432067E0680121A6
S31508002670A9408843E060E0680121A9400843E0607A
S31508002680012080032840002803D0012000F020F80C
S3150800269007E00120C0032840002802D0012000F0EE
S315080026A017F8F0BD002905D08268FF2301331A43C5
S315080026B0826004E08268FF2301339A438260704790
S315080026C000210160416081600173016141617047C9
S315080026D0002806D0064949680C221143044A51606D
S315080026E005E0034949680C229143014A5160704745
S315080026F00024014010B524480078012834D1002070
S31508002700214908702149088012E0204800884000C5
S315080027101F49085A1F490988C9001F4A89181B4AB0
S3150800272012885200885219480088401C17490880A8
S31508002730164800880428E8DB7E2002F09FFB02206A
S3150800274000F02EF901211548FFF7ACFF1148008863
S31508002750401C1049088008460088142804DB00201D
S31508002760088001200E4908700D480078002806D018
S31508002770FFF78AFE00200A49087000F059FC7E20FF
S3150800278002F07CFB10BD0000840100209E010020A1
S31508002790B4040020A0010020EC040020002401401D
S315080027A07C010020FFB583B00C46029400200190FE
S315080027B0002726E000261CE0721C039951430846B0
S315080027C0791CFFF7A7F80546A54201D9281B00E0A2
S315080027D0601B05460298A84204D90295059806701A
S315080027E0069807700298002802D10120019002E09D
S315080027F0761C402EE0D300BF0198002800D002E0E6
S315080028007F1C042FD6D300BF029807B0F0BD000086
S3150800281000BF00BF00BF00BF00BFBFF34F8F00BFA0
S3150800282000BF00BF06480749C86000BF00BF00BF19
S31508002830BFF34F8F00BF00BF00BF00BF00BFFDE75B
S315080028400400FA0500ED00E010B500F001F810BD2F
S3150800285010B523480078002817D1224801F00EF950
S3150800286001283CD11F480078002838DD1D4800782B
S31508002870402834DC01F03EFF1B4908600120184956
S31508002880087000201949087029E0164A174909787E
S31508002890491C501801F0F2F8012816D1134800789F
S315080028A0401C124908700F4800780978884216D1EA
S315080028B000200B4908700B484078FF280FD10B48B9
S315080028C0007802280BD1FFF7A3FF01F013FF064992
S315080028D009686431884202D900200149087010BD90
S315080028E049010020700400204C0100204801002006
S315080028F010B586B004460121880301F037F8012196
S31508002900480401F013F801220921C80600F031FB3A
S3150800291001220A210920C00600F02BFB01A801F0BC
S31508002920ECFF0194302168460181002141818181B3
S3150800293001821821C18101A9184801F09BFF0121D4
S31508002940164801F074FF05A800F069FB0121490249
S3150800295068468182012181751821C17505A909205A
S31508002960C00600F0B9FA0121890268468182482129
S31508002970C17505A90920C00600F0AEFA1B216846F4
S315080029800170032141700121817000F09BFF012233
S315080029900221024801F063FF06B010BD003801406D
S315080029A001B506490098086002E07E2002F066FA42
S315080029B0024800680028F8D108BD0000540100202C
S315080029C0014600220E4B1A61CA005A6100229A611A
S315080029D005221A6100BF0A4A1069C207D20F002AE7
S315080029E004D0012212040240002AF4D0044A1269D3
S315080029F052085200024B1A6100229A617047000081
S31508002A0000E000E010B500210448FFF74BFE022065
S31508002A1000F04AF801200249087010BD0024014060
S31508002A208401002000B589B00121084600F07EFF28
S31508002A301A4800F045F801A800F08EF818480190E9
S31508002A4018480290002168460173042004906846DD
S31508002A500175802141754900C182890001832021C1
S31508002A608176090281830021C183018401A90B486B
S31508002A7000F04CF80121094800F01CF80122022157
S31508002A80064800F039F809216846017002214170AC
S31508002A900121817000F016FF09B000BD0800024050
S31508002AA000240140B4040020014948607047000032
S31508002AB0000002400268520852000A43026070474A
S31508002AC010B50446206840084000206000202060B9
S31508002AD06060A060E060E1B2084608380521FEF7AC
S31508002AE019FF01460F2088400249496808430149F1
S31508002AF0486010BD00000240002A03D003680B435B
S31508002B00036002E003688B430360704710B50A7AD6
S31508002B108B7D1A430B7C1A434B7C1A434B8A1A4308
S31508002B208B8A1A430B8B1A434B8B1A430368094C3F
S31508002B3023401A43026002680123DB039A438B8B06
S31508002B401A430260CA6842600A6882604A68C260BC
S31508002B5010BD00000F80FFFF002101604160017277
S31508002B60C160017441744182818281750183418308
S31508002B708183704770B506460C4621460A4800F020
S31508002B804BF90546002D01D1401E70BD0648854209
S31508002B9002D10648051B00E02D1B22462946304671
S31508002BA0FEF7E2FE2046F0E700F4000800FC000805
S31508002BB070B506460C4621460A4800F02DF905462A
S31508002BC0002D01D1401E70BD0648854202D1064837
S31508002BD0051B00E02D1B224629463046FEF7C4FE9B
S31508002BE02046F0E700F0000800F8000870B5064631
S31508002BF00C4621460A4800F00FF90546002D01D17A
S31508002C00401E70BD0648854202D10648051B00E0F5
S31508002C102D1B224629463046FEF7A6FE2046F0E73B
S31508002C2000F800080000010870B505460C46224663
S31508002C300249284600F0B1F8204670BD00F40008A5
S31508002C4070B505460C4622460249284600F0A5F806
S31508002C50204670BD00F0000810B504460848006913
S31508002C600221084306490861084644610069402173
S31508002C70084303490861034800F00EF910BD000037
S31508002C8000200240FF0F00000C48C068C007C00FB4
S31508002C90002801D0012070470848C0680421084070
S31508002CA0002801D00220F6E70448C0681021084031
S31508002CB0002801D00320EEE70420ECE700200240BC
S31508002CC003480069802108430149086170470000EC
S31508002CD00020024030B504460D460548006901212A
S31508002CE008430349086125800F2000F0D5F830BD58
S31508002CF00020024010B57E2002F0C0F8064800F019
S31508002D000FF87E2002F0BAF8044800F009F87E2091
S31508002D1002F0B4F810BD000000F4000800F0000846
S31508002D2010B5044600F0ACF82046FFF795FFFFF70C
S31508002D30C7FF10BD70B503460125002208E0500004
S31508002D401C5A0748844201D0002506E0501C82B26E
S31508002D50CE0F761876109642F1DC00BF284670BD75
S31508002D60FFFF0000F8B505460E46144600F088F841
S31508002D707E2002F083F8002707E029883046FFF70F
S31508002D80A9FFB61CAD1C781C87B2E10F09194910BA
S31508002D90B942F2DCFFF794FFF8BDF8B507460C46D2
S31508002DA015462946204600F037F80646002E0DD16E
S31508002DB02046FFF7B5FF012080022018FFF7B0FF75
S31508002DC02A4621463846FFF7CDFF24E00120800237
S31508002DD02018401BB0420AD1012080022018FFF7B4
S31508002DE09FFF2A4631463846FFF7BCFF13E001200D
S31508002DF0C0022018401BB04208D12046FFF790FFBA
S31508002E002A4631463846FFF7ADFF04E02A463146E2
S31508002E103846FFF7A7FFF8BDF8B505460E462F4614
S31508002E20E807C00F002801D000BFFEE731460120A1
S31508002E30C002FEF785FD002901D000BFFEE7002489
S31508002E400BE020467043471931463846FFF772FFB4
S31508002E50012800D108E0601C84B231460120C00276
S31508002E60FEF76EFDA042ECDC00BF31460120C00231
S31508002E70FEF766FDA04200D100273846F8BD0000DF
S31508002E80024803494860034848607047230167457C
S31508002E9000200240AB89EFCD10B5024600BFFFF710
S31508002EA0F3FE0346521EFF2400E0641E002CFCD1EC
S31508002EB0012B01D1002AF2D10648006977218843FF
S31508002EC0044908613420C860002A01D1052010BDD4
S31508002ED01846FCE700200240F8B50246CD782F07D1
S31508002EE03F0FCD7810263540002D01D08D782F4321
S31508002EF01446002011E085062B0E0D880126864013
S31508002F003540002D07D025680F269E40B5433E461E
S31508002F109E4035432560451CE8B20828EBDB141DA6
S31508002F200D882D120095002011E085062B0E01252F
S31508002F308540009E3540002D07D025680F269E4007
S31508002F40B5433E469E4035432560451CE8B20828F1
S31508002F50EBDBCD78282D04D155690E8835435561AC
S31508002F6006E0CD78482D03D115690E8835431561DD
S31508002F70F8BD70B54D07EB0E082902DA054620356F
S31508002F8001E0054624352C460F269E402568B543A4
S31508002F9016469E403543256070BD000038B5044688
S31508002FA00D460920C006844203D10121480400F0D9
S31508002FB0BDFC1148844203D10121000200F0B6FC91
S31508002FC00E48844203D10121000200F0AFFC0C48F0
S31508002FD0844203D10121080500F0A8FC684600F0E8
S31508002FE01EF868460580012181700021C170694676
S31508002FF02046FFF771FF38BD000400480008004866
S31508003000000C0048024690680840002801D00120BC
S3150800301070470020FCE74161704701617047002155
S31508003020C9430180022181700421C17070470000E4
S3150800303000B591B000200F900E900D900C907E2058
S3150800304001F01CFF002010901FE010984000FE4978
S31508003050085A0590FEF71DFFFC490690FEF73EFD4F
S315080030600790FEF78BFF0022F94B09910890FEF7AF
S3150800307025FE0B910A90FEF7A9FF10998900F54ADB
S3150800308050501098401C80B2109010980428DCDB31
S31508003090F0488068F0490690FEF720FD0790FEF795
S315080030A06DFFEE4AEE4B09910890FEF7FFFD0B9176
S315080030B00A90FEF78BFF0F90E6484068E6490690AF
S315080030C0FEF70CFD0790FEF759FFE44AE44B099119
S315080030D00890FEF7EBFD0B910A90FEF777FF0E902E
S315080030E00F98FEF74BFF0022D94B05910490FEF787
S315080030F0DDFD09910890DB480F99FEF7B2FC0590B3
S31508003100FEF73CFF07910690099B089AFEF73EFEDC
S315080031100B910A90FEF75AFFD34908600E98FEF7FE
S315080031202DFF0022CA4B05910490FEF7BFFD0991B9
S315080031300890CC480E99FEF794FC0590FEF71EFF02
S3150800314007910690099B089AFEF720FE0B910A90B4
S31508003150FEF73CFFC5490860C548808D322830DA3D
S31508003160C448408B0190FEF7AFFEC34AC34B039198
S315080031700290FEF7A3FD0022C14B05910490FEF7CD
S3150800318005FE09910890BB48408B0290FEF781FE28
S31508003190BC490390FEF7A2FC0490B3480168049862
S315080031A0FEF75BFC0590FEF7E9FE07910690099B82
S315080031B0089AFEF7EBFD0B910A90FEF707FF0D90B4
S315080031C05CE0AB48808DBE282CDAAA48408B069076
S315080031D0FEF75FFE0890A748808B0590FEF759FE1C
S315080031E0A9490690FEF77AFC07900899FEF739FC7C
S315080031F0A4490990FEF772FC0B909E48408B0790F5
S31508003200FEF747FE9F490890FEF768FC0990964826
S3150800321001680998FEF721FC0A900B99FEF75EFCF7
S315080032200D902BE09348408B0690FEF732FE0890EF
S315080032309048008C0590FEF72CFE93490690FEF701
S315080032404DFC07900899FEF70CFC8E490990FEF78D
S3150800325045FC0B908748408B0790FEF71AFE894974
S315080032600890FEF73BFC09907F4801680998FEF72D
S31508003270F4FB0A900B99FEF731FC0D907C48C08D43
S31508003280322830DA7B48008B0190FEF71DFE7A4A19
S315080032907A4B03910290FEF711FD0022784B0591B7
S315080032A00490FEF773FD099108907248008B02900E
S315080032B0FEF7EFFD73490390FEF710FC04906B4888
S315080032C001680498FEF7C9FB0590FEF757FE0791BB
S315080032D00690099B089AFEF759FD0B910A90FEF78E
S315080032E075FE0C905CE06248C08DBE282CDA6148F9
S315080032F0008B0690FEF7CDFD08905E48C08B0590C2
S31508003300FEF7C7FD60490690FEF7E8FB07900899A7
S31508003310FEF7A7FB5B490990FEF7E0FB0B905548C3
S31508003320008B0790FEF7B5FD56490890FEF7D6FBC9
S3150800333009904E4801680998FEF78FFB0A900B9989
S31508003340FEF7CCFB0C902BE04A48008B0690FEF764
S31508003350A0FD08904748408C0590FEF79AFD4A491B
S315080033600690FEF7BBFB07900899FEF77AFB4549DE
S315080033700990FEF7B3FB0B903E48008B0790FEF7CB
S3150800338088FD40490890FEF7A9FB0990374801686F
S315080033900998FEF762FB0A900B99FEF79FFB0C90C3
S315080033A03A480D99FEF704FB0B90FEF7B4FD384931
S315080033B0086036480C99FEF7FBFA0B90FEF7ABFD52
S315080033C0344908602A48808D314909684018C00385
S315080033D0010C27488185C08D2E4909684018C0030D
S315080033E0010C2348C1851B48C0682B490A90FEF783
S315080033F038FB0B90FEF78FFD81B21D488187FF3899
S31508003400C1380088FF21F531884272DD002019494C
S315080034106C3908800F4800680990FEF7AFFD024630
S315080034200B460B910A901DA001F078FD094800682B
S315080034300990FEF7A3FD1B4A1B4B0B910A90FEF75A
S31508003440B1FD57D2034831E07401002000F07F45F2
S3150800345000000840DC040020000040412506819554
S31508003460438BD43F000048438C0100209001002084
S31508003470CC03002078020020091B9E5E29CB703FF2
S3150800348000408F4000007A44002474490000C84177
S3150800349094010020980100200000C84225660D0A04
S315080034A000000000736891ED7C3FDD3F00680990DD
S315080034B0FEF764FD2F4A304B0B910A90FEF772FD1A
S315080034C012D240212D48FFF79DFD00280CD12C482B
S315080034D04078012808D12A48C078002804D129490B
S315080034E0486006212648C170012025492031087206
S315080034F014E03CE02448006824490B90FEF78CFD54
S315080035000CD21F482030C07C002803D11C4920312A
S31508003510087203E001201A49203108721A48006827
S315080035201B490B90FEF778FD04D20120144920317F
S31508003530487203E0002012492031487210482030B2
S31508003540007A00280ED10E484078012804D10102DD
S315080035500A48FFF760FD0AE0FF2101310748FFF737
S315080035605CFD04E0FF2101310448FFF756FD11B068
S3150800357000BD00009CC420B07268D13F000400481A
S315080035800C0400200C020020DC0400206F12233FEC
S31508003590333313400148806A70470000C0F7FF1FA5
S315080035A00148C06A70470000C0F7FF1F014800685D
S315080035B0704700005801002003480068034909784D
S315080035C04018014908607047580100206001002032
S315080035D008B50121480400F0A9F90121880400F082
S315080035E0A5F96846FFF71BFD0121C9036846018056
S315080035F04821C17069460920C006FFF76DFC684678
S31508003600FFF70DFD01210903684601804821C170B5
S3150800361069460920C006FFF75FFC6846FFF7FFFC0E
S315080036204021684601800421C17069460148FFF7B8
S3150800363053FC08BD0004004810B50121C903092040
S31508003640C006FFF7DFFC002869D177488079002893
S315080036505AD175484078012837D173482030C07C44
S31508003660002832D171480078401C70490870084615
S31508003670007805281CDB0020087004216C48FFF739
S31508003680CCFC694894384089002807D169486A49BA
S315080036904860012164489438418106E00020664963
S315080036A04860002160489438418101F007FC0CE02D
S315080036B05E480078022808DC5F4840687D210901D9
S315080036C0884202D900205C49486057482030C07CAF
S315080036D0002816D15848406D5849884211D3524897
S315080036E094384089002805D1554853494865002033
S315080036F0486006E04D480078022802DC00204E4962
S3150800370048600121484881714E48007800280DD14B
S3150800371001204C49087001214348817006E00020C9
S315080037204849087000214048817081714248C06844
S315080037304049884272D900203F49C86000213A486A
S3150800374081702030C07C002862D108213848FFF7F4
S3150800375064FC35489438408803285FDA3248943840
S31508003760408900285AD130484038C08D5A280FDA87
S315080037702D482030407A00280AD12B484078012865
S315080037804CD129492031C87400202B49486045E0AE
S3150800379025484078012802D1002027494860224858
S315080037A04038C08D5A282ADB27484088274988424E
S315080037B003DC25488088884208DD1B48C078002835
S315080037C004D11D49486005211748C1701E48408824
S315080037D00A2803DB1C4880880A2808DA1248C078B9
S315080037E0002804D11449486004210F48C1700E48C6
S315080037F0C078002812D102210B48C1700EE00A4891
S315080038002030407A012809D101210748C17005E016
S315080038100020094948600021034841707E2001F0D4
S315080038202DFB0148807810BD0C040020C400002040
S3150800383000040048DC0500000C020020307500007A
S31508003840606D0000A201002074010020E60F000050
S3150800385008B50121480400F069F80121880400F040
S3150800386065F86846FFF7DBFBFF210E3168460180E5
S31508003870012181701021C17069461148FFF72CFBA0
S31508003880B62168460180012181701021C170694600
S315080038900920C006FFF720FB10210920C006FFF704
S315080038A0BAFB80210920C006FFF7B5FB01210448B1
S315080038B0FFF7B1FB08210248FFF7AFFB08BD000080
S315080038C0000400488178002925D0174903221202EE
S315080038D08918027892109200895802789207D30EB6
S315080038E0FF229A40914342789207120E03789B076B
S315080038F0DB0E9A4011430C4A03231B02D2180378A5
S315080039009B109B00D1500178CA06D20E0121914026
S31508003910054A116007E00178CA06D20E01219140D6
S31508003920014A80321160704700E100E0002905D0A5
S31508003930054A52690243044B5A6104E0024A526935
S315080039408243014B5A61704700100240002905D096
S31508003950054AD2690243044BDA6104E0024AD26995
S315080039608243014BDA61704700100240002905D0F6
S31508003970054A92690243044B9A6104E0024A926935
S315080039808243014B9A6170470010024010B500F05F
S3150800399031F804494968F02211400909024A515C84
S315080039A0C84010BD001002402201002010B5FFF7E4
S315080039B0EDFF05494968072212021140090A034A20
S315080039C0515CC84010BD00000010024022010020D2
S315080039D010B5FFF7DBFF054949680722D2021140F7
S315080039E0C90A034A515CC84010BD000000100240D5
S315080039F022010020F8B51E4840680C21084004281A
S31508003A0002D008282ED101E01A4C2DE01848403083
S31508003A100069C007C00F00280AD015484030006961
S31508003A2002210840002801D0134802E0114800E0AE
S31508003A30104807460E4840300069FF21090408402F
S31508003A40000C451C0A484030006907210902084055
S31508003A50000A461C3946694308463146FDF75AFFAF
S31508003A60044601E0034C00BF00BF2046F8BD000035
S31508003A700010024000127A0000093D0070B50446A5
S31508003A8000250221074800F0D8FE002808D005487E
S31508003A9000F02CFF20700221024800F0C6FE012526
S31508003AA0284670BD0038014010B500F001F810BD79
S31508003AB000B585B06248006801210843604908607E
S31508003AC000BF5F480068022108400028F9D05D4819
S31508003AD05D4908605D480068102108435B49086035
S31508003AE008460068C008C000086057490968481EAB
S31508003AF05749FDF70FFF0490544800680499490791
S31508003B00490F0843514908604D48406851490840E3
S31508003B104B49486008464068902108434849486030
S31508003B20084640684860484800684649884207D9B8
S31508003B3043484068052109020843414948600BE0AB
S31508003B40414800684449884206D93D4840680121F1
S31508003B50890208433A4948606B4601AA3A4801680F
S31508003B603E48FEF71FFE3648403000698008800050
S31508003B703349403108610846006940084000086139
S31508003B80684600784007400F02906846007940066C
S31508003B90400E03902A48C069890508432849C86128
S31508003BA02748403000692E490840254940310861B8
S31508003BB0039800040299090208432149403109691A
S31508003BC008431F49403108611D480068012109065C
S31508003BD008431B49086000E000BF19480068012136
S31508003BE0490608400028F7D0154840688008800034
S31508003BF0134948600846406802210843104948604E
S31508003C0000E000BF0E4840680C2108400828F8D19B
S31508003C100120FEF7D5FE0A48406810218843084966
S31508003C2048600120FEF7CCFE05484068802188439D
S31508003C30034948600120FEF7C3FE05B000BD000039
S31508003C400010024000A24A0434010020002002406D
S31508003C5000366E010FC0FFFF0051250200127A00E0
S31508003C60FFF800FF042806D1064909690422114312
S31508003C70044A116105E00349096904229143014A8E
S31508003C801161704700E000E010B5FFF795FC9C480D
S31508003C900088401C9A49088008464068401C4860CD
S31508003CA098480088401C974908809748006800286B
S31508003CB004D095480068401E934908609348807868
S31508003CC0012805D18E48C068401C8D49C86002E0AD
S31508003CD000208B49C8608D482030807B012805D19B
S31508003CE087484069401C8649486102E000208449AB
S31508003CF0486186480079012805D18148006C401C36
S31508003D007F49086402E000207D4908647C494868C8
S31508003D100A21FDF7FFFD002927D17C482030C0780D
S31508003D207A4920318978884207DD784820308078BA
S31508003D30401C76492031887017E074482030C078D6
S31508003D40724920318978884200D10EE06F482030C8
S31508003D50C0786E4920318978884206DA6B48203067
S31508003D608078401E69492031887068482030C07CB8
S31508003D70022804D065482030C07C032804D1604856
S31508003D80806B401C5E498863604820304079002873
S31508003D900AD15E482030C07C042805D15848806C7A
S31508003DA0401C5749886402E00020554988645748F2
S31508003DB02030C07C002803D151490865C86426E034
S31508003DC05248C079012805D14D48006D401C4C4920
S31508003DD0086502E000204A4908654C48007A01282F
S31508003DE012D14748C06C401C4549C8644748203032
S31508003DF08079002804D108468068401C886006E05F
S31508003E0000203F49886002E000203D49C8643F48D9
S31508003E102038807F04280AD13948406D3C498842B9
S31508003E2008D23748406D401C3549486502E00020F5
S31508003E3033494865012109030920C006FFF7E2F85E
S31508003E40002813D031482030007A00280ED12F4898
S31508003E50407801280AD12A48806D2E49884208D21E
S31508003E602748806D401C2649886502E000202449C1
S31508003E70886526482030807A01280AD12048C06DF6
S31508003E802549884208D21E48C06D401C1C49C86591
S31508003E9002E000201A49C8651C482030007B01282A
S31508003EA005D11748006E401C1549086602E0002037
S31508003EB01349086615482030407B012805D110486B
S31508003EC0406E401C0E49486602E000200C494866D0
S31508003ED07E2000F0D3FF40211048FFF793F8002812
S31508003EE00AD00748806E0E49884208D20448806E78
S31508003EF0401C0349886602E000200149886610BD17
S31508003F000C02002050010020540100200C0400205F
S31508003F1050C3000088130000701700000004004812
S31508003F20B888000010B516480068012108431449EE
S31508003F300860084640681349084011494860084621
S31508003F400068114908400E490860084600680121C2
S31508003F50890488430A49086008464068C321090459
S31508003F6088430749486008460068084908400449E4
S31508003F7008609F2000048860FFF796FD10BD0000CA
S31508003F80001002400CC0FFF8FFFFF6FEFFFF8F008F
S31508003F9008B501214804FFF7C9FC022201210920BE
S31508003FA0C006FEF7E6FF0221684601801821C170A7
S31508003FB00121817069460920C006FEF78DFF01219F
S31508003FC04804FFF7B3FC022211460920C006FEF793
S31508003FD0D0FF0421684601801821C1700121817033
S31508003FE069460920C006FEF777FF08BD30B587B0D9
S31508003FF004460D4601210846FFF7A8FC04A800F070
S3150800400033F9059468460582002101838176817417
S3150800401004A90120800700F0F1F8684600F0D2F8FC
S31508004020602168460170012141700020019000213D
S315080040306846017269460120800700F057F869460C
S315080040400120800700F08AF80821C80600F07EF8EB
S315080040500821C80600F0B0F84021080600F038F834
S315080040604021080600F03CF80121880700F00AF80C
S315080040700121880700F01EF80121880700F00EF8D4
S3150800408007B030BD002904D0026880231A430260B5
S3150800409003E0026880239A4302607047002904D02F
S315080040A0026801231A43026003E0026852085200BC
S315080040B002607047002905D0426C0123DB031A43CE
S315080040C0426404E0426C0123DB039A43426470476E
S315080040D0826907231B039A430B021A4382617047BE
S315080040E0C26970239A430A43C261704710B5826950
S315080040F007231B039A430B781B021A4382610A7A29
S3150800410012014B781B011A43036A3024A3431A434E
S3150800411002624A6882630C4A904213D14A7A1201B3
S315080041208B781B011A43036AC024A3431A4302620D
S315080041304A8992008B899B001A4343682401A3434A
S315080041401A43426010BD0000002C01408269012319
S31508004150DB029A430B021A438261704710B5C269A3
S3150800416070239A430B781A43C2610A7A12024B7873
S315080041701B021A43036A03242402A3431A43026256
S315080041804A68C2630B4A904213D14A7A12028B7864
S315080041901B021A43036AA400A3431A4302624A890C
S315080041A012018B891B011A434368A400A3431A43CF
S315080041B0426010BD002C0140C26908239A430A4395
S315080041C0C2617047002101704170817041600172BF
S315080041D0417241818181704701229207904201D143
S315080041E0816301E08AB28263704701229207904296
S315080041F001D1C16301E08AB2C26370470268032332
S315080042001B029A430B891A430260134A904206D04E
S3150800421001229207904202D0104A904205D10268C4
S3150800422070239A438B781A4302600B4A904205D052
S315080042300B4A904202D00B4A904205D1026B120AF1
S3150800424012028B7A1A4302634A68C2620A88826239
S315080042500122426170470000002C01400004004022
S3150800426000440140004801400021C9434160002143
S3150800427001800181817081727047000010B50024A9
S31508004280FA48807B00280FD1F9484068F94909683F
S31508004290401AF94988420BD90021F4482038417060
S315080042A00020F249C87403E0F1484068F149086003
S315080042B0EE48C07A030000F072FE050478F1EFEECE
S315080042C0ED00EA4920390A8CE9494868B32105F026
S315080042D0E1FC0446E5482038C08B912805DA0F2210
S315080042E00121002002F09CFD04E000220121104675
S315080042F002F096FDDD482038008CB42809D0DB484A
S315080043002038008CB32804D0D8482038008CB5282B
S3150800431013D1D6486038C08DD8490988884208D054
S315080043200020D249487308466038C08DD3490880B2
S3150800433006E00120CD49487302E00020CB494873C6
S31508004340CB48406ECE49884226D9C8482038C08B0B
S31508004350801ECC490988884216DCC4482038C08BA0
S31508004360801CC849098888420EDBC6480088A528EB
S315080043700FDB03F0A5FA0120BC49C8720020BC492E
S315080043804866C149087004E0B8482038C08BBD4962
S3150800439008800020B64948660020BC4908702246B5
S315080043A00121084602F03CFD9CE1B04920398A8B80
S315080043B0AF494868B32105F06DFC04460022012187
S315080043C0084602F02DFDA9482038808BB42809D06C
S315080043D0A6482038808BB32804D0A4482038808B80
S315080043E0B52813D1A1486038808DA4490988884228
S315080043F008D000209D49487308466038808D9F493B
S31508004400088006E001209949487302E00020974990
S3150800441048739748406E9A49884222D9934820386B
S31508004420C08B801E97490988884212DC8F4820383D
S31508004430C08B801C9349098888420ADB03F0D8FAA6
S3150800444002208A49C8720020894948668E49087040
S3150800445004E086482038C08B8A49088000208449B1
S3150800446048668A48007800280ED180482038008C93
S31508004470822805DD00220121104602F0D1FC08E061
S3150800448001208249087004E022460121002002F03A
S31508004490C7FC27E125E107E16BE0FFE7734920390F
S315080044A00A8C73494868E52105F0F4FB04460022A6
S315080044B00121104602F0B4FC6C482038008CE6282E
S315080044C009D06A482038008CE52804D06748203887
S315080044D0008CE72813D165486038C08D674909887C
S315080044E0884208D000206149487308466038C08D64
S315080044F06249088006E001215C48417302E0002118
S315080045005A4841735A48406E5D49884228D95748E7
S315080045102038C08B801E5B490988884218DC5348BE
S315080045202038C08B801C57490988884210DB5548BB
S315080045300088D22811DB03F0F3FA03204B49C8722E
S3150800454003F08AF900204A4948664F49087004E092
S3150800455046482038C08B4B490880002044494866A5
S3150800456000204B49087022460121084602F058FCF3
S31508004570B8E03E4920398A8B3D494868E52105F06F
S3150800458089FB044600220121084602F049FC374807
S315080045902038808BE6280BD034482038808BFF21C2
S315080045A02C31884204D031482038808BE72813D133
S315080045B02E486038808D31490988884208D0002005
S315080045C02A49487308466038808D2C49088006E0D9
S315080045D001202649487302E00020244948732448EC
S315080045E0406E2749884231D920482038C08B801E22
S315080045F024490988884221DC1C482038C08B801C45
S3150800460020490988884219DB1E480088B4281ADB25
S315080046101C480088D22816DA03F01AFB042013492E
S31508004620C87203F019F90122FE21572004F08DF90A
S3150800463000200F4948661449087004E00B482038E2
S31508004640C08B104908800020094948661048007840
S31508004650002823D105482038C08BC8281ADD002237
S315080046600121104602F0DCFB1DE000002C040020AE
S315080046700C02002010010020C409000016010020C9
S31508004680DC0500000C010020F800002018010020BD
S315080046901901002001201449087004E0224601216E
S315080046A0002002F0BDFB1DE010494868FF21F531E6
S315080046B0FDF730F9002913D100200C4948660C494A
S315080046C048850122FE21572004F03FF900220121E6
S315080046D0104602F0A5FB00220121084602F0A0FBC5
S315080046E000E000BF00BF10BD190100200C02002029
S315080046F04004002010B5FEF759FF10BD70B5FFF74E
S3150800470045F905467D21C900FDF704F90446601EF2
S315080047100C49884200D90CE0601E0B494861032108
S31508004720081F00F04BFC0020074988610720086134
S3150800473000BF0420FFF796FA0021481E00F03EFC51
S3150800474070BD0000FFFFFF0000E000E010B5022189
S31508004750144800F07BF8002822D0124800F0C6F86A
S31508004760C4B21148C07F022813D10F482030007800
S31508004770002811D10D488079AA2805D10B48C471A3
S315080047800121094820300170AA2C05D107488471F7
S3150800479002E0204603F0F4FA0221024800F045F848
S315080047A010BD000000380140EC0300209C050020E5
S315080047B010B504462146054800F09CF800BF0121C3
S315080047C0024800F03AF80028F9D010BD0038014038
S315080047D070B505460E4600247E2000F04FFB00BF4C
S315080047E020E0042C19DD701EA04216DD285D7E2807
S315080047F006D17D20FFF7DCFF5E20FFF7D9FF0FE02B
S31508004800285D7D2805D1FFF7D3FF5D20FFF7D0FF90
S3150800481006E0285DFFF7CCFF02E0285DFFF7C8FF3A
S31508004820601C84B2B442DCDB70BD416170478269AA
S31508004830520852000A43826170470246906808404F
S31508004840002801D0012070470020FCE70246D06806
S315080048500840002801D0012070470020FCE7002A04
S3150800486003D003690B43036102E003698B430361C9
S315080048707047000070B504460D460026E0693021F1
S31508004880884329790843E061E06944218843A97986
S315080048900843E061E06980088000297A0843E061FE
S315080048A0A0691821884369890843A061A069042181
S315080048B08843297B0843A0610B48844203D1FFF74C
S315080048C087F8064602E0FFF771F80646304629687B
S315080048D0FDF720F80009206230462968FDF71AF826
S315080048E00007000F606270BD003801400146486845
S315080048F0C0B27047CAB2026070474B21C901016055
S315080049003021017100218171017218214181002134
S315080049100173704710B51C484088030000F03FFB40
S315080049200504111E292A2B0017485430808FFF21B1
S315080049301B31884204DA01211348418000F0BEFA8F
S3150800494019E011485430808FFF210531884204DA76
S3150800495002210D48418000F0B1FA0CE00A485430B3
S31508004960808FF62804DA03210748418000F0A6FA6A
S3150800497001E000E000BF00BF0348943040780028FB
S3150800498001D100F09BFA10BD7803002010B57548D8
S315080049904088002806D0012845D0022871D003286F
S315080049A040D199E002216F487430817740216E48E2
S315080049B0FEF728FB002827D06C494868FF21F53107
S315080049C0FCF7A8FFC007C00F00280ED180210920D8
S315080049D0C006FEF722FB01216348FEF71EFB1021E5
S315080049E00920C006FEF719FB1CE080210920C00635
S315080049F0FEF711FB01215C48FEF70DFB102109208B
S31508004A00C006FEF708FB0DE080210920C006FEF768
S31508004A1004FB01215448FEF700FB10210920C006BB
S31508004A20FEF7FBFA9BE001214E487430817740215E
S31508004A304D48FEF7E7FA002813D04C494868FF218D
S31508004A40F531FCF767FFC007C00F002804D1012124
S31508004A504548FEF7E2FA08E001214348FEF7DBFA8B
S31508004A6003E001214048FEF7D8FA80210920C00654
S31508004A70FEF7D1FA10210920C006FEF7CCFA6EE03F
S31508004A80FFE740213848FEF7BDFA002815D0374918
S31508004A904868FF21F531FCF73DFFC007C00F002825
S31508004AA005D180210920C006FEF7B5FA0AE0802163
S31508004AB00920C006FEF7B1FA04E080210920C006E5
S31508004AC0FEF7ABFA01212848FEF7A5FA10210920BE
S31508004AD0C006FEF7A0FA42E040212348FEF792FA04
S31508004AE0002815D021494868FF21F531FCF712FF47
S31508004AF0C007C00F002805D180210920C006FEF78F
S31508004B008AFA22E080210920C006FEF786FA1CE010
S31508004B1016494868CD21FCF7FDFEC007C00F0028DE
S31508004B2005D180210920C006FEF775FA0DE00F4968
S31508004B304868CD21FCF7EEFEC007C00F002804D058
S31508004B4080210920C006FEF768FA01210648FEF70B
S31508004B5062FA10210920C006FEF75DFA00BF00BF01
S31508004B6010BD000078030020000400480C02002055
S31508004B7010B5A948807F030000F011FA05044680A5
S31508004B80C4F4F300A4482038808FFF2116318842E8
S31508004B9003DB0121A048817735E09F482038808FC4
S31508004BA0FF210C3188420ADD9B4874384088022868
S31508004BB005D0022198487438418000F07FF94021D9
S31508004BC09648FEF71FFA00281DD095494868FF2128
S31508004BD0F531FCF79FFEC007C00F002805D18021DC
S31508004BE00920C006FEF717FA04E080210920C0064E
S31508004BF0FEF713FA10210920C006FEF70CFA012168
S31508004C008648FEF708FA05E183482038808FFF2199
S31508004C102731884203DB02217F4881772DE0402136
S31508004C207E48FEF7EFF9002827D07D494868FF211E
S31508004C30F531FCF76FFEC007C00F002804D101212B
S31508004C407648FEF7E8F903E001217448FEF7E5F92E
S31508004C5080210920C006FEF7DEF910210920C006CA
S31508004C60FEF7D9F96C4874384088012805D0012127
S31508004C7069487438418000F021F9CBE0664820384D
S31508004C80808FFF212831884203DB03216248817720
S31508004C9037E040216148FEF7B5F9002831D0604970
S31508004CA04868FF21F531FCF735FEC007C00F00281C
S31508004CB00ED180210920C006FEF7AFF90121574819
S31508004CC0FEF7ABF910210920C006FEF7A6F90DE09C
S31508004CD080210920C006FEF79EF910210920C0068A
S31508004CE0FEF799F901214D48FEF795F94A487438B7
S31508004CF04088002805D0002147487438418000F0D4
S31508004D00DDF887E040214548FEF77CF9002843D0C6
S31508004D10012109030920C006FEF774F9002807D007
S31508004D203F48806D3F49884202D904213A48817735
S31508004D303B494868FF21F531FCF7ECFDC007C00F79
S31508004D40002810D180210920C006FEF766F9012146
S31508004D503248FEF762F910210920C006FEF75DF910
S31508004D600FE056E019E080210920C006FEF753F946
S31508004D7010210920C006FEF74EF901212748FEF743
S31508004D804AF9254874384088002805D00021224869
S31508004D907438418000F092F83CE040211F48FEF745
S31508004DA031F9002834D01C4874384088002805D0CA
S31508004DB0002119487438418000F080F81848406D81
S31508004DC0194988420ED280210920C006FEF725F926
S31508004DD001211248FEF721F910210920C006FEF725
S31508004DE01CF90DE080210920C006FEF714F91021F0
S31508004DF00920C006FEF70FF901210848FEF70BF94E
S31508004E0005484030007A012802D1032102488177FB
S31508004E1000E000BF00BF10BDEC03002000040048FE
S31508004E200C020020941100003075000003488068C9
S31508004E30400840000149886070470000002C004087
S31508004E4080210143014A116070470000002C004090
S31508004E5003488068002801D0012070470020FCE73D
S31508004E60002C004010B5FFF7F3FF002804D0FFF729
S31508004E70DDFF662000F002F810BD00004106490E6D
S31508004E80014A116070470000002C00400449496837
S31508004E90FF22813291430143014A51607047000065
S31508004EA0002C004004494968C909C9014206520E46
S31508004EB01143014A51607047002C004010B57E200E
S31508004EC0FFF7DCFF0948FDF72BFF094909488185EB
S31508004ED006212C3000F025FD06492C318881402218
S31508004EE0024904482C30FDF758FF10BD00F80008A9
S31508004EF0FBAA00004C03002070B505460C460121AC
S31508004F00C802FEF723FDFF208130FFF7BFFF2046CA
S31508004F10FFF7C8FF2846FFF793FF70BD0FB410B51B
S31508004F2003A9044B044A029800F054F910BC08BCC3
S31508004F3004B018479D780008040200200FB41CB579
S31508004F400246002007AC00290BD0491E01910092A9
S31508004F50064B6A462146069800F03CF9009A00215D
S31508004F6011701CBC08BC04B0184700000D59000895
S31508004F702021020C01D010211046020A01D0104649
S31508004F800839020901D01046091F820801D01046C7
S31508004F90891E420801D0881E7047081A704730B427
S31508004FA07446641E2578641CAB4204D3635D5B00BB
S31508004FB0E31830BC18471D46F8E7000010B500286E
S31508004FC019DB1A4A03231B02D21883089B00D258FE
S31508004FD08307DC0EFF23A3409A438B071B0E840727
S31508004FE0E40EA3401A43114B032424021B19840818
S31508004FF0A4001A5118E00E4A03071B0F083B9B082A
S315080050009B00D2588307DC0EFF23A3409A438B07E5
S315080050101B0E8407E40EA3401A43054B0407240F0E
S31508005020083CA408A4001A5110BD000000E100E0E5
S315080050301CED00E002E008C8121F08C1002AFAD1D8
S3150800504070477047002001E001C1121F002AFBD1FA
S3150800505070470000014908607047000008020020F8
S31508005060F0B51FB486B00998089A030D00210243CB
S3150800507014D05148514A181850430514119801285C
S3150800508010981AD0281A401C00264D4F4D490096F4
S3150800509001910490002812DA444211E01198012483
S315080050A049A3012801D11098C1430698119A846032
S315080050B00360C26041600BB0F0BD4042E4E70446BD
S315080050C0210500203F4A001C51410391029012E03D
S315080050D0E00707D032463B4601990098FCF7EEFDFB
S315080050E00191009032463B4610461946FCF7E6FD0C
S315080050F006460F466410002CEAD10498039B002844
S31508005100029A0999089806DAFCF7D8FD019B009AD5
S31508005110FCF7D4FD05E0FCF739FE019B009AFCF785
S3150800512035FE04460E460022284BFDF7F5F803D84F
S315080051300020C043014607E00022254B20463146A1
S31508005140FCF70AFDFDF7C8F8102409E0002C0ADB75
S315080051500A220023FCF76AFF079B30321A55641EA1
S3150800516002460A43F2D11122641C079B121B1C1922
S31508005170119B012B03D0012308430ED10AE00843F3
S3150800518004D0112010900020119077E71098151A76
S315080051906D1E0BE01098824202DD00236D1C03E0B1
S315080051A0824201DA00236D1E002BEED00698119973
S315080051B08260C16030C07EE701FCFFFF104D000031
S315080051C0000014400000F03F300000000000F043EB
S315080051D00000E03FFFB597B00646002518E22528EF
S315080051E077D100242746FD49049400E00443761C41
S315080051F032780120203A90400842F7D130782A28A0
S315080052000ED00222307801463039092916D8049979
S315080052100A235943303940181443761C0490F1E7A1
S31508005220189802C804911890002904DA012040034E
S3150800523004434842049002200443761C30782E2802
S3150800524014D1042004437078761C2A2809D11898AA
S31508005250761C80C8189009E00A214F43303FC719C9
S31508005260761C3078014630390929F5D930786C280A
S3150800527010D006DC4C281AD068280ED06A2817D118
S3150800528004E0742813D07A2812D110E001204005D2
S3150800529004430CE00121090501E0032109050C433B
S315080052A07178814203D1012000052418761C761CEA
S315080052B03078119066280BD013DC58287DD009DC8D
S315080052C000287BD04528F6D04628F4D047281AD19E
S315080052D0A5E118E0632835D0642870D0652812D176
S315080052E09DE170286CD008DC6728F1D069287BD04E
S315080052F06E280DD06F2806D1BAE073282ED07528EF
S3150800530071D0782859D01A9A199990476D1C7EE160
S315080053106002400F022809D003280DD004281898E7
S3150800532001680DD00D60001D189070E11898EA17F5
S3150800533001680D604A60F6E7189801680D80F2E783
S315080053400D70F0E718986A4601781172001D1890DA
S315080053500020507202A80090012005E0189802C8A3
S31508005360189000200091C04361070DD5002101E087
S315080053700199491C0191B94212DA8142F8DB009A77
S31508005380515C0029F4D10BE0002101E00199491C88
S3150800539001918142FADB019A0099895C0029F5D1CD
S315080053A0019904981A9B471A21463846199A00F01B
S315080053B097FA0199401945180BE04FE02CE113E0E4
S315080053C04EE0009800990078491C00911A9A19999C
S315080053D090470198401E0190401CF2D1214638465C
S315080053E01A9B199A10E137E00A20002100900191D2
S315080053F06002410F022907D0189A01CA1892C217EB
S315080054009446032908D00AE01898C01DC108C900A7
S3150800541005C91891944607E000B2C21794460429B4
S3150800542002D140B2C1178C4600226146944506DA7D
S315080054300A460021404291418C462D2102E0210571
S3150800544004D52B216A461173012103E0E10701D037
S315080054502021F7E7029155E00A200AE0102008E02B
S31508005460102000900021042004430191082703E03E
S3150800547008200021019100906002410F022907D0FF
S31508005480189A01CA189200229446032908D008E0FF
S315080054901898C01DC108C90005C91891944603E0AB
S315080054A080B2042900D1C0B200210291210729D572
S315080054B01199702906D0009A1021019B4A401A4377
S315080054C005D00EE040216A461173012108E06146C5
S315080054D0014306D030216A4611731199517302218E
S315080054E00291009A0821019B4A401A430AD1614653
S315080054F0014301D1610705D530216A46117301219F
S315080055007F1E02911199582904D035A10E910DA933
S315080055100D910DE037A1F9E76146019B009AFCF76A
S3150800552085FD0E9B8C469B5C0D9A521E0D92137040
S3150800553061460143F0D10D9805A9081A203001905B
S31508005540600703D501200004844300E00127019881
S31508005550874201DD381A00E00020019900904118C1
S31508005560029809180498401A0490E00306D42146C4
S315080055701A9B199A049800F0B3F94519002706E012
S3150800558003A81A9AC05D199990476D1C7F1C02984A
S315080055908742F5DBE0030CD521461A9B199A049835
S315080055A000F09EF9451904E01A9A30201999904797
S315080055B06D1C0099481E00900029F5DC08E00D983E
S315080055C00D990078491C0D911A9A199990476D1CE6
S315080055D00199481E01900029F1DC63E109280100C0
S315080055E0303132333435363738396162636465664B
S315080055F0000000003031323334353637383941420D
S31508005600434445460000000000F05AF94519761C47
S315080056103078002800D0E2E528461BB0F0BD6007C8
S3150800562000D406271898C01DC108C90048680A682A
S315080056300831C30FDB071891190001D09CA108E0B7
S31508005640210501D59BA104E0E10701D09AA100E05C
S315080056509AA1430011985B08109165280CD006DCC6
S31508005660452809D046281DD0472841D141E066285B
S3150800567018D067283CD13CE00021112F01DB11200E
S3150800568000E0781C0191009008A911A8FFF7E8FC32
S31508005690139905910021119A15927F1C129801976A
S315080056A0009150E00120C00703900120019008A94D
S315080056B0009711A8FFF7D4FC139A149905920022B3
S315080056C0119B009212981593059A0192002901D010
S315080056D0104602E0791C40180190381A01D5019845
S315080056E004E04042401E0090781C0190C01B0290C6
S315080056F043E0012F00DA01270021112F01DD1120D7
S3150800570000E038460191009008A911A8FFF7A8FC07
S3150800571013990591119A00211298159200910197F3
S3150800572021070CD40599B94201DB019900E00191E2
S31508005730012904DD159A491E515C302906D0B84264
S3150800574001DA011D05DA0121029115E00199491EC8
S31508005750EDE7002805DC0099411800910199091A1E
S3150800576003E0019A411C914200DD01910099401A1B
S31508005770401C02900120C0070390200706D4029916
S315080057800198814202DB0020C0430290002069464E
S31508005790C87707AF012103980337C907884224D081
S315080057A0022011902B201290039800280CDA404210
S315080057B003902D20129007E00A210398FCF7AAF817
S315080057C030317F1E039039701199481E11900029B7
S315080057D0F2DC03980028EFD1791E12980870307809
S315080057E0202108404530BF1E387006A8C01BC01DC2
S315080057F0039010980078002800D0012001994118DC
S315080058000298C0170918039809180498401A401EE8
S315080058100490E00306D421461A9B199A049800F0CE
S315080058205FF8451910980078002803D01A9A199934
S3150800583090476D1CE00324D521461A9B199A0498B3
S3150800584000F04EF845191CE00098002807DB00997F
S315080058500598884203DD1598405C199901E0199965
S3150800586030201A9A904700986D1C401C00900298A8
S31508005870401E0290002804D11A9A2E2019999047A2
S315080058806D1C0199481E01900029DDDC05E0387879
S315080058901A9A7F1C199990476D1C0399481E039004
S315080058A00029F4DC21461A9B199A0498ACE60000F4
S315080058B02D0000002B000000200000000000000062
S315080058C0F8B5044600251E461746880404D405E0A4
S315080058D039462020B0476D1C641EF9D52846F8BD08
S315080058E0FFB50446002581B01E46C80301D53027FA
S315080058F000E02027880404D505E038460399B04718
S315080059006D1C641EF9D5284605B0F0BD4A68002A04
S3150800591006D00A68531C0B6010704868401E486021
S31508005920704710B502460023002901D1002010BD9A
S3150800593003E01488921CE01883B208464C1EA1B2F4
S315080059400028F6D11846F2E710B5C0484078002876
S3150800595064D110210920C006FDF75DFB80210920CE
S31508005960C006FDF758FB0121B948FDF754FB002096
S31508005970B6492031C874002301221946184603F097
S3150800598019FA00231A461946184603F013FAB148BD
S315080059904068FF21F531884204D20421AC48FDF75E
S315080059A03CFB51E10421AA48FDF735FBA9484068AC
S315080059B0A9498842F5D9A5488079002817D1A5486C
S315080059C040687D214901884201D2FEF7A3FF0821DC
S315080059D09F48FDF720FB00219C48C17000209B4989
S315080059E02031487188719B49486248630CE0402120
S315080059F09748FDF707FB002806D00021934820307A
S31508005A00C17401212038417020210920C006FDF704
S31508005A1002FB7D2040018F49486015E18B48203004
S31508005A20C07C0300FFF7BBFA060471B5FEFDFC70E7
S31508005A300020864920314871887186494862486342
S31508005A40002301221946184603F0B4F900231A4622
S31508005A501946184603F0AEF97C484038C18D818650
S31508005A602030C07F012809D17A4840697B4988429D
S31508005A7003D9002175482038C17710BD754840689C
S31508005A807D210901884227D90020754908706F4889
S31508005A908079002802D16F49486002E071486D4953
S31508005AA0486040216A48FDF7ADFA00280CD1FEF798
S31508005AB031FF08216648FDF7AEFA7E20FFF7DEF9CA
S31508005AC01E20FCF76DFF02E00020624948600421B1
S31508005AD05F48FDF7A0FA17E020210920C006FDF768
S31508005AE09CFA08215A48FDF798FA5A484068FF2157
S31508005AF0F531884208D9554894384089002803D199
S31508005B0004215348FDF787FA9DE052484068FF2173
S31508005B10F531884204D204214D48FDF77EFA03E0A8
S31508005B2004214B48FDF777FA48482038C07F0528F6
S31508005B3017D100220121084601F072F9434840387E
S31508005B40818D4030408B814205DA64220121002094
S31508005B5001F066F907E000220121104601F060F91C
S31508005B6001E0FEF78BFB39484038C18D4030408B49
S31508005B7081420DDB35484038818D4030408B81426B
S31508005B8006DB002033494860022030492031C874BA
S31508005B9059E030484068FF21F531884204D2042193
S31508005BA02B48FDF73AFA03E004212948FDF733FAB2
S31508005BB0284840682C4988421ED92448408BD22858
S31508005BC01AD12248008CCF2812DB2048008CD52811
S31508005BD00EDA01201D49203108731E48006E1F4940
S31508005BE0884209D90122FE21672002F0AEFE03E0B1
S31508005BF0002016492031087314482038C07F05282C
S31508005C001BD100220121084601F00AF90F48403845
S31508005C10818D4030408B814209DA3C22012102E025
S31508005C2010E00EE00CE0002001F0FAF807E0002290
S31508005C300121104601F0F4F801E0FEF71FFB02E02F
S31508005C4001E000E000BF00BF00BF16E70C0400201B
S31508005C50000400480C020020B80B0000881300005E
S31508005C60C4000020C40900001027000010B5BE4873
S31508005C704078002864D110210920C006FDF7CBF929
S31508005C8080210920C006FDF7C6F90121B748FDF7AE
S31508005C90C2F90020B4492031C874002301221946EC
S31508005CA0184603F087F800231A461946184603F0E3
S31508005CB081F8AF484068FF21F531884204D20421B3
S31508005CC0AA48FDF7AAF94DE10421A848FDF7A3F96A
S31508005CD0A7484068A7498842F5D9A348807900288B
S31508005CE017D1A34840687D214901884201D2FEF7B1
S31508005CF011FE08219D48FDF78EF900219A48C170CA
S31508005D000020994920314871887199494862486349
S31508005D100CE040219548FDF775F9002806D00020CB
S31508005D2091492031C87401218F48417020210920EA
S31508005D30C006FDF770F97D2040018D49486011E1E4
S31508005D4089482030C07C0300FFF729F9060475B29C
S31508005D50FEFDFC74002084492031487100218248E8
S31508005D60203081710020824948624863002301225D
S31508005D701946184603F01EF800231A46194618460F
S31508005D8003F018F878484038C18D81862030C07FE6
S31508005D90012809D1764840697749884203D9002104
S31508005DA071482038C17710BD714840687D210901C6
S31508005DB0884227D90020714908706B4880790028E5
S31508005DC002D16B49486002E06D4869494860402144
S31508005DD06648FDF717F900280CD1FEF79BFD082148
S31508005DE06248FDF718F97E20FFF748F81E20FCF7F1
S31508005DF0D7FD02E000205E49486004215B48FDF7B4
S31508005E000AF917E020210920C006FDF706F908213E
S31508005E105648FDF702F956484068FF21F531884291
S31508005E2008D9514894384089002803D104214F489D
S31508005E30FDF7F1F895E04E484068FF21F5318842B4
S31508005E4004D204214948FDF7E8F803E0042147484D
S31508005E50FDF7E1F844482038C07F062817D100220C
S31508005E600121104600F0DCFF3F484038C18D403024
S31508005E70408B814205DA50220121084600F0D0FF06
S31508005E8007E000220121084600F0CAFF01E003F0FE
S31508005E9053FE35484038C18D4030408B814206DB81
S31508005EA000203349486002202F492031C87458E041
S31508005EB02F484068FF21F531884204D204212B4837
S31508005EC0FDF7ABF803E004212848FDF7A4F82848B5
S31508005ED040682C4988421ED92348408BD2281AD1BB
S31508005EE02148008CCF2812DB1F48008CD5280EDAF3
S31508005EF001201D49203108731D48006E1E4988423D
S31508005F0009D90122FE21672002F01FFD03E00020C7
S31508005F1015492031087314482038C07F06281AD13D
S31508005F2000220121104600F07BFF0F484038C18D42
S31508005F304030408B814208DA3C220121084600F0B5
S31508005F406FFF0AE00CE00AE008E00022012108469B
S31508005F5000F066FF01E003F0EFFD02E001E000E07B
S31508005F6000BF00BF00BF1EE70C0400200004004865
S31508005F700C020020B80B000088130000C4000020A3
S31508005F80C40900001027000010B56E4840780028A4
S31508005F9064D110210920C006FDF73DF880210920AB
S31508005FA0C006FDF738F801216748FDF734F80021E7
S31508005FB064482030C174002301221946184602F0AD
S31508005FC0F9FE00231A461946184602F0F3FE5F4802
S31508005FD04068FF21F531884204D204215A48FDF76A
S31508005FE01CF8ACE004215848FDF715F857484068F6
S31508005FF057498842F5D953488079002817D153481C
S3150800600040687D214901884201D2FEF783FC0821B8
S315080060104D48FDF700F800214A48C170002049495B
S315080060202031487188714949486248630CE040212B
S315080060304548FCF7E7FF002806D0002141482030F4
S31508006040C17401212038417020210920C006FCF7BF
S31508006050E2FF7D2040013D49486070E03948203024
S31508006060C07C002804D0012866D0022866D164E0E6
S31508006070002134482030417100203249203188718E
S315080060803249486248632F484038C18D818620309E
S31508006090C07F012809D12D4840692E49884203D975
S315080060A0002128482038C17710BD284840687D213E
S315080060B00901884227D90020274908702148807994
S315080060C0002802D12149486002E024481F49486057
S315080060D040211D48FCF796FF00280CD1FEF71AFC54
S315080060E008211948FCF797FF7E20FEF7C7FE1E20F9
S315080060F0FCF756FC02E000201449486004211248C7
S31508006100FCF789FF17E020210920C006FCF785FF68
S3150800611008210D48FCF781FF0C484068FF21F5313E
S31508006120884208D9074894384089002803D10421B1
S315080061300548FCF770FF01E000E000BF00BF00BFA4
S31508006140B2E700000C040020000400480C020020FE
S31508006150B80B000088130000C4000020C409000022
S31508006160F0B587B00020069005900024002504901D
S3150800617000260027F748807B012814D1F648406995
S315080061804B21C90088420ED90020F2498873F2498A
S315080061904861F2490880F2490870FF210131EF4849
S315080061A0801DFBF7FAFBEB482038007801286CD1F4
S315080061B07E20FEF763FEE948C0790002E749097ABE
S315080061C008430690E548407A0590E448847AC67AFA
S315080061D00246117B507B01F027FF0746DF4AD17A3A
S315080061E0107B01F021FF05460021DA4820380170AE
S315080061F00121203081730020D7494861D94A069881
S31508006200811A904242D03CDCD74A811A90423ED04D
S315080062101EDCD64A811A90423AD010DCD44A811A3A
S31508006220904236D006DC442861D0D249401800286E
S3150800623071D19CE201296FD00229F9D1D1E2012955
S315080062406BD002296AD0032969D01029F0D153E30B
S315080062502A297DD00CDC22297BD004DC012979D0BF
S315080062601129E5D1FCE3232975D02929E0D15DE080
S31508006270312971D0332970D044296FD05729D7D105
S315080062809CE0881E282846D204E0EAE376E095E3F7
S31508006290C1E27AE243007B449B885B009F446A0024
S315080062A0660072003B003B003B003B003B003B00A6
S315080062B03B003B003B003B003B003B003B003B00F8
S315080062C021020D024F022B0274018501D5013B0004
S315080062D03B003B004000300148019C01BA013B00ED
S315080062E03B009F00AB00F7001101C500DF000598D1
S315080062F0062809D1A048007800280BD102F050FBE7
S3150800630001209D49087005E00598062802DD012050
S3150800631002F046FB12E2FDE34BE288E29CE2C7E2AA
S315080063200022FE21E82002F010FBF3E789496039D4
S31508006330898F0A2251430846FBF7A0FD8F49009032
S31508006340FBF7CCFB8E490190FBF78BFB029006E02E
S31508006350D0E3A3E386E3B7E318E0EAE3F8E3FBF761
S31508006360DAFD80B2039002F0C4FAD3E7032002F004
S3150800637017FBCFE7042002F013FBCBE7052002F05A
S315080063800FFBC7E7022002F00BFBC3E7012C0AD17B
S3150800639071486C30008B0123002297210090FE2063
S315080063A002F073FA09E06C486C30408B0223002235
S315080063B097210090FE2002F068FAABE704217148A5
S315080063C0FCF72BFEC820FCF7EBFA04216D48FCF716
S315080063D022FE0022FE21BD2002F0B7FAF3E35D4853
S315080063E0C07C002806D05B486038828DC18D0020AD
S315080063F002F0DCF9E7E3002C0AD156486038C08D74
S3150800640000231A46F0210090FE2002F03EFA0BE027
S31508006410012C09D14F486038808D01230022F021D4
S315080064200090FE2002F031FACDE3002C0AD14A484A
S315080064306C30408800231A46F3210090FE2002F0B3
S3150800644024FA0BE0012C09D143486C3080890123DA
S315080064500022F3210090FE2002F017FAB3E3002C85
S3150800646003D13D486C30458002E03B486C3085815D
S3150800647039486C308089FF21F531884206DA01F007
S31508006480EBF90022FE21F42002F05FFA9BE3002CD0
S315080064900AD131486C30808800231A46F1210090D1
S315080064A0FE2002F0F2F90BE0012C09D12A486C30E3
S315080064B0C08901230022F1210090FE2002F0E5F9AF
S315080064C081E3002C03D124486C30858004E0012C3C
S315080064D002D121486C30C5811F486C308088FF2165
S315080064E0F53188420BDC1C486C30C089884206DCD2
S315080064F001F0B2F90022FE21F22002F026FA62E348
S31508006500002C0AD114486C30C08800231A46E921A9
S315080065100090FE2002F0B9F909E0012C07D11920F4
S3150800652001230022E9210090FE2002F0AEF94AE399
S31508006530002C02D108486C30C580FF202D308542DA
S3150800654006DA01F089F90022FE21EA2002F0FDF9B7
S3150800655039E300002C0400200C0200209C050020D2
S31508006560F1010020CBFE000066FE000055FE00008B
S3150800657052FE0000AF01FFFF000200200000A0400D
S315080065800000E04000040048002C0CD1F7480089C0
S315080065906421484380B200231A46E2210090FE2077
S315080065A002F073F900E000BF0DE3002C06D1642168
S315080065B02846FBF7C5F981B2EC480181EB4800890A
S315080065C0FF21F531884206DC01F046F90022FE215A
S315080065D0E32002F0BAF9F6E2002C0CD1E348408930
S315080065E06421484380B200231A46EB210090FE201E
S315080065F002F04BF90DE0012C0BD1DC48008A64212E
S31508006600484380B201230022EB210090FE2002F0CD
S315080066103CF9D8E2002C07D164212846FBF790F90B
S3150800662081B2D248418108E0012C06D1642128466E
S31508006630FBF786F981B2CD48018201F00DF90022F7
S31508006640FE21EC2002F081F9BDE2012C19D1C848DF
S31508006650408803280BDAC6484089002807D101215B
S31508006660C348B430C1740020C0496C394860002260
S31508006670FE21E42002F069F90121BD4894304170F9
S315080066801AE0002C13D10021B9489430417000203B
S31508006690B749B431C8740022FE21E42002F055F946
S315080066A00020B4490870B1496C39486004E00022FA
S315080066B0FE21E42002F049F985E2002C0FD1AE480C
S315080066C0C07A32280CDCAC48C17AA848418201F06D
S315080066D0C3F80022FE21DF2002F037F900E000BFF0
S315080066E071E2A248408A00231A46DE210090FE2065
S315080066F002F0CBF867E2002C0FD19F48C07A322807
S315080067001CDC9D48C17A9948818201F0A5F80022CF
S31508006710FE21E12002F019F910E0012C0ED196486D
S31508006720C07A32280ADC9448C17A9048C18201F0BE
S3150800673093F80022FE21E12002F007F943E2002C3B
S3150800674009D18A48808A00231A46E0210090FE2053
S3150800675002F09BF80AE0012C08D18448C08A01237C
S315080067600022E0210090FE2002F08FF82BE28349F8
S315080067707E488183C1830184418401F06DF800223B
S31508006780FE21512002F0E1F81DE2002C10D1002E66
S3150800679003D17748943087830AE0012E03D17448E1
S315080067A09430C78304E0022E02D1714894300784DE
S315080067B009E2002C14D1FCF7EDFE04900498000CB5
S315080067C000231A4653210090FE2002F05EF8049832
S315080067D080B20123002253210090FE2002F055F8D2
S315080067E0F1E1002C0AD16148C08B00905F48838B89
S315080067F000225421FE2002F00EF80BE0012C09D1EC
S315080068005A48408C00905948038C01225421FE2096
S3150800681002F001F8D7E1002C08D101215448743060
S31508006820C177002202215648FEF719F8CBE1002C61
S3150800683011D1FF2101315048801DFBF7AEF8002029
S315080068404D49088002214A487430C1770022FE214A
S31508006850562002F07AF8B6E1002C19D100214448F6
S31508006860B430C1720020444908800321404874307E
S31508006870C1770121203041702030C17400203B4986
S315080068806C3948600022FE21572002F05EF80EE0BF
S31508006890012C0CD1002136487430C17700203449C8
S315080068A0B431C8740122FE21572002F04EF88AE15D
S315080068B0002C18D100202E49B431C8722E49088000
S315080068C004212B487430C1770121203041702030D3
S315080068D0C174002025496C3948600022FE215820E1
S315080068E002F033F807E0012C05D100212048743066
S315080068F0C1774030C17466E1002C1BD100201E49C7
S31508006900088006211A487430C17701212030417069
S3150800691001201749B431C874002014496C394860FD
S31508006920B4211348943041830022FE21652002F0E9
S315080069300CF842E0012C25D100200F4908800621D9
S315080069400B487430C1770121203041702030C17462
S31508006950002006496C394860D221054894304183A5
S315080069600022FE21652001F0F0FF26E078020020D3
S3150800697078030020000200209C0500200410000077
S3150800698000380140022C18D10020904908800621C1
S315080069908F48C17701212030417001208C49403150
S315080069A0C87400208B494860F0218948203041830B
S315080069B00022FE21652001F0C8FF04E1002C19D150
S315080069C000208249088005218148C17701212030AD
S315080069D0417001207E494031C87400207D494860D5
S315080069E0B4217B48203041830022FE21662001F035
S315080069F0ACFF34E0012C19D1002074490880052128
S31508006A007348C17701212030417001207049403117
S31508006A10C87400206F494860D2216D4820304183F0
S31508006A200022FE21662001F090FF18E0022C16D104
S31508006A3000206649088005216548C1770121203074
S31508006A4041702030C174002062494860F0216048D6
S31508006A50203041830022FE21662001F076FFB2E055
S31508006A6006E0B1E000215A48C1774030C174AAE077
S31508006A70002C08D107215648C1770022FE2177202D
S31508006A8001F063FF09E0012C07D100215048C177C6
S31508006A900122FE21772001F058FF94E0002C12D144
S31508006AA064220121002000F0BBF9002201210846DA
S31508006AB000F0B6F9012046494031C8740022FE218B
S31508006AC0882001F042FF7EE0002C12D164220121C9
S31508006AD0084600F0A5F900220121104600F0A0F9A9
S31508006AE001203B494031C8740022FE21892001F06B
S31508006AF02CFF68E0384939480068FAF7B2FF019078
S31508006B00FBF709FA80B23449039035480068FAF76A
S31508006B10A8FF00E056E00190FBF7FDF980B202906D
S31508006B200398009000229021FE20029B01F073FE3C
S31508006B3049E0002C33D1002E0BD126486C30C78390
S31508006B400022FE21522001F000FF00F085FE26E01B
S31508006B5026E0012E0AD11F486C30878300F07CFEA0
S31508006B600122FE21522001F0F0FE18E0022E0AD181
S31508006B7018486C30478400F06FFE0222FE2152202E
S31508006B8001F0E3FE0BE0032E09D112486C300784AE
S31508006B9000F062FE0322FE21522001F0D6FE12E02A
S31508006BA0002C0ED101200A494031C8740121084839
S31508006BB020304170012006494031C873002005493C
S31508006BC0486000E000BF00BF07B0F0BD9C0500208C
S31508006BD0EC0300200C02002000007A4490010020FB
S31508006BE08C010020F0B589B0002008900790069027
S31508006BF05148007801287DD150488079AA287AD151
S31508006C004E48C079322877DA4C48C079002873DDB7
S31508006C104A49C97908461938FBF730F9089008989F
S31508006C20FBF7ACF90646464A464BFBF747F80446D7
S31508006C300022454BFAF790FF0391029043480068FB
S31508006C40FBF79CF901910090039B029AFBF79EF8CB
S31508006C5005910490FBF7BAF907900898FBF78EF9A7
S31508006C600446374A374BFBF729F80022364B019181
S31508006C700090FAF771FF0391029035480068FBF718
S31508006C807DF90646039B029AFBF780F80591049066
S31508006C90FBF79CF906902F490798FBF7B3F938D20A
S31508006CA02D490798FBF7B8F933D22A490698FBF716
S31508006CB0A9F92ED228490698FBF7AEF929D2274911
S31508006CC00798FAF7CEFE0446FBF725F981B2244861
S31508006CD0418322490698FAF7C4FE0446FBF71BF9D6
S31508006CE081B21F48018300F0B7FD1D48408B009014
S31508006CF01B4802E01DE019E014E0038B0022602126
S31508006D00FE2001F088FD0122FE21562001F01DFE1D
S31508006D1004E00022FE21562001F017FE0021064855
S31508006D202038C177002104482038C177002102485D
S31508006D30017009B0F0BD00000C0400209C0500207D
S31508006D40091B9E5E29CB703F0000F03F8C01002096
S31508006D5090010020000018410000E04000007A443D
S31508006D60780200202A494A88498A511A814209DB51
S31508006D7027496C398968264A6C3AD1620021254A26
S31508006D8011701BE022494988814217DC214909789C
S31508006D90002913D120498A8F40318A8201211D4A50
S31508006DA011701B496C398968194A6C3AD26A891A72
S31508006DB0174A6C3A516211468968516314498A88A0
S31508006DC0898A511A814209DB0021144A1170104937
S31508006DD06C3989680E4A6C3A116318E00C4989883F
S31508006DE0814214DC0D490978002910D10A498A8F95
S31508006DF04031CA820121094A117005496C398968EE
S31508006E00034A6C3A126B891A014A6C3A91627047C6
S31508006E1078020020E4000020CC030020E5000020D2
S31508006E2070B505460E461446002E02D0012E4AD1EC
S31508006E3020E0002D02D0012D1AD10CE0602101209E
S31508006E408007FDF745F9002101208007FDF7C4F901
S31508006E501E4804700CE0602101208007FDF740F908
S31508006E60002101208007FDF7C0F91948047000BF0A
S31508006E7000BF28E0002D02D0012D22D110E01348D2
S31508006E800078A0420BD0602101208007FDF720F989
S31508006E90214601208007FDF79FF90C48047010E091
S31508006EA00B480078A0420BD0602101208007FDF72F
S31508006EB017F9214601208007FDF797F90448047061
S31508006EC000BF00BF00BF00BF70BD0000A3010020C7
S31508006ED0A401002010B5F3484078012879D1F1487B
S31508006EE02030407C0028F9D1EE48C0780300FEF730
S31508006EF056F80805075DB0FDFCFBFAF9002010BD41
S31508006F00E9494868FF219131FAF704FD8007800FA7
S31508006F10002809D180210920C006FCF77CF8012148
S31508006F20E248FCF778F83AE0DF494868FF219131F2
S31508006F30FAF7F0FC8007800F012809D18021092083
S31508006F40C006FCF76AF80121D848FCF764F826E081
S31508006F50D5494868FF219131FAF7DCFC8007800F94
S31508006F60022809D180210920C006FCF754F801211E
S31508006F70CE48FCF750F812E0CB494868FF2191311A
S31508006F80FAF7C8FC8007800F032808D10121C748F3
S31508006F90FCF743F880210920C006FCF73CF81021CD
S31508006FA00920C006FCF737F80120A8E7BE4948685B
S31508006FB0C821FAF7AFFC8007800F00280AD1802184
S31508006FC00920C006FCF727F80121B848FCF723F882
S31508006FD038E065E1B4494868C821FAF79BFC8007A0
S31508006FE0800F012809D180210920C006FCF715F871
S31508006FF00121AE48FCF70FF824E0AB494868C821E0
S31508007000FAF788FC8007800F022809D18021092019
S31508007010C006FCF700F80121A448FBF7FCFF11E0C5
S31508007020A1494868C821FAF775FC8007800F03282C
S3150800703008D101219D48FBF7F0FF80210920C006F1
S31508007040FBF7E9FF10210920C006FBF7E4FF012042
S3150800705055E795494868C821FAF75CFC8007800F10
S31508007060002809D180210920C006FBF7D4FF012199
S315080070708E48FBF7D0FF3DE08B494868C821FAF7F0
S3150800708049FC8007800F012809D180210920C00604
S31508007090FBF7C3FF01218548FBF7BDFF2AE08249BC
S315080070A04868C821FAF736FC8007800F022809D1FC
S315080070B080210920C006FBF7AEFF01217B48FBF7BC
S315080070C0AAFF17E078494868C821FAF723FC800721
S315080070D0800F03280ED101217448FBF79EFF8021FB
S315080070E0092004E0DBE0B2E05FE034E009E0C00636
S315080070F0FBF791FF10210920C006FBF78CFF012042
S31508007100FDE669494868FF212D31FAF703FCC007F7
S31508007110C00F002805D180210920C006FBF77BFF98
S315080071200EE061494868FF212D31FAF7F3FBC007E5
S31508007130C00F002804D080210920C006FBF76DFF88
S3150800714010210920C006FBF766FF01215748FBF707
S3150800715062FF0120D3E654494868FF219131FAF7C6
S31508007160D9FBC007C00F002805D180210920C00619
S31508007170FBF751FF0EE04C494868FF219131FAF7B9
S31508007180C9FBC007C00F002804D080210920C0060B
S31508007190FBF743FF10210920C006FBF73CFF01213E
S315080071A04248FBF738FF0120A9E63F494868C8214D
S315080071B0FAF7B0FB8007800F002809D18021092043
S315080071C0C006FBF728FF01213848FBF724FF37E004
S315080071D035494868C821FAF79DFB8007800F0128C2
S315080071E009D180210920C006FBF717FF01212F4886
S315080071F0FBF711FF24E02C494868C821FAF78AFBF7
S315080072008007800F022809D180210920C006FBF7D4
S3150800721002FF01212548FBF7FEFE11E022494868D6
S31508007220C821FAF777FB8007800F032808D10121C8
S315080072301E48FBF7F2FE80210920C006FBF7EBFE8D
S3150800724010210920C006FBF7E6FE012057E616497D
S315080072504868C821FAF75EFBC007C00F002805D1A9
S3150800726080210920C006FBF7D6FE0DE00E494868C6
S31508007270C821FAF74FFBC007C00F002804D08021A9
S315080072800920C006FBF7C9FE10210920C006FBF736
S31508007290C2FE01210548FBF7BEFE01202FE600BF0E
S315080072A000BF2CE60C0400200C0200200004004855
S315080072B010B5FE48C07C002874D0FC486038C08DE4
S315080072C0FF217D31884204DCF8486038808D884289
S315080072D01CDDF6482038C078002817D1F4484088C5
S315080072E00A2813DDF2484088F24988420EDAF04847
S315080072F080880A280ADDEE488088884206DA002057
S31508007300ED4948600321E9482038C170EA48006C15
S31508007310EA4988420AD9E5482038C078002805D1C4
S31508007320E54948600321E1482038C170DF48C07C40
S31508007330042838D1DD48407900282BD1DB4820388D
S31508007340C07901281ED1DC48006DDD49884231D953
S315080073500020D9490865D5486038418E808D81421C
S315080073600BDBD2482038C078002823D1D2494860A0
S315080073700721CE482038C1701CE0CC486038818D82
S31508007380418617E00020CC490865C8486038818DD9
S3150800739041860FE00020C8490865C4486038818DD9
S315080073A0418607E028E00020C3490865BF486038E1
S315080073B0818D4186BD48C07C01282BD1BB48203829
S315080073C0007A01281ED1BC48C06CBD49884228D91C
S315080073D00020B949C864B5486038018EC08D81421D
S315080073E00BDBB2482038C07800281AD1B249486069
S315080073F00721AE482038C17013E0AC486038C18D0B
S3150800740001860EE00020AC49C864A8486038C18DE2
S31508007410018606E00020A849C864A4486038C18DE2
S315080074200186A24820384078012877D19F4820381D
S31508007430C07800280BD0002301221946184601F00F
S31508007440B9FC00231A461946184601F0B3FC9748BA
S315080074502038C0780300FDF7A2FD0805073C71A493
S31508007460D8FDFCFB002010BD93484068E121C90007
S31508007470884229D910210920C006FBF7CCFD8021B6
S315080074800920C006FBF7C7FD01218E48FBF7C3FD9F
S315080074900120864948740846C07B002807D18649DA
S315080074A048600021814820384170C17008E0824850
S315080074B04068AF210901884202D900207E49486008
S315080074C001207A49087402E00020784948740120AE
S315080074D0C9E7794840687C4988422AD91021092099
S315080074E0C006FBF798FD80210920C006FBF793FD2F
S315080074F001217448FBF78FFD01206C494874084642
S31508007500C07B00280BD16C494860002167482038A9
S315080075104170C1700020684948600DE02BE166485B
S315080075204068AF210901884206D9002062494860AF
S3150800753002E000205D494874012094E75E484068EF
S315080075406249884228D910210920C006FBF763FD45
S3150800755080210920C006FBF75EFD01215948FBF78B
S315080075605AFD0120514948740846C07B00280AD1B3
S315080075705149486000214D4820384170C1700020AB
S315080075804D4948600BE04C4840685149884206D945
S3150800759000204949486002E0002044494874012017
S315080075A061E7454840687D210901884228D91021AC
S315080075B00920C006FBF72FFD80210920C006FBF72E
S315080075C02AFD01213F48FBF726FD0120374948746B
S315080075D00846C07B00280AD137494860002133484D
S315080075E020384170C1700020334948600BE03248AA
S315080075F040683349884206D900202F49486002E08E
S3150800760000202A49487401202DE72B484068E121CB
S31508007610C90088422DD910210920C006FBF7FBFCBA
S3150800762080210920C006FBF7F6FC01212548FBF757
S31508007630F2FC01201D4948740846C07B00280ED17B
S315080076401D4948600021194820384170C17002E080
S3150800765090E05CE012E00020174948600CE016480C
S315080076604068AF210901884206D9002012494860BE
S3150800767002E000200D4948740120F4E60E484068EF
S315080076801349C83988423CD910210920C006FBF79E
S31508007690C2FC80210920C006FBF7BDFC0121094870
S315080076A0FBF7B9FC01200149487413E02C040020BB
S315080076B074010020E60F00000C0200207011010082
S315080076C0B80B000000040048A4060000C409000026
S315080076D0AC0D00000846C07B002809D12749486040
S315080076E0002127484170C1700020244948600CE0F9
S315080076F0224840682349884207D900201F49486024
S3150800770003E000211E48203041740120ABE61B48E7
S3150800771040681D49884227D910210920C006FBF771
S315080077207AFC80210920C006FBF775FC0121174861
S31508007730FBF771FC0121124820304174C07B0028F8
S3150800774009D10E49486000210D484170C1700020DA
S315080077500A4948600CE0094840680D49884207D93B
S3150800776000200649486003E0002005492031487496
S31508007770012078E600BF00BF75E600000C02002075
S315080077800C040020CC100000A406000000040048E9
S315080077908C0A000010B5052421E080212C48FAF750
S315080077A0FCF880212A48FBF7E5F912212848FEF75C
S315080077B0B8F82749898C88420CD125482C38808D01
S315080077C02449884204D000F0E9FC00F045F800E0BE
S315080077D010BD04E0002000E0401C8028FCDB2046A9
S315080077E0611ECCB20028D8D100BF052423E0802131
S315080077F01748FAF7D2F880211548FBF7D9F912216C
S315080078001348FEF78EF81249898C88420ED1104823
S315080078102C38808D0F49884204D000F0BFFC00F058
S315080078201BF802E000F018F8D2E704E0002000E0B8
S31508007830401C8028FCDB2046611ECCB20028D6D12D
S3150800784000BF00F0ABFC00F007F800BFC0E700007F
S3150800785078020020FBAA000010B57E20FDF70EFB7B
S31508007860FBF748FA0B490C48818512212C30FEF7A4
S3150800787058F809492C318884802107482C30FBF7B1
S31508007880D3F97E20FDF7FAFA802103482C30FBF75E
S31508007890D7F910BDFBAA00004C02002070B50446BB
S315080078A00D46E1B20548FDF725F800BF012103485A
S315080078B0FCF7C3FF0028F9D0204670BD0038014008
S315080078C0F0B587B000240020069005904049088B43
S315080078D0FAF7DFFA07463F49FAF700F905463C4941
S315080078E0088BFAF7D6FA3B490490FAF7F7F80746F1
S315080078F0394801683846FAF7B0F806462946FAF7CD
S31508007900EDF806903549088CFAF7C3FA0646344965
S31508007910FAF79FF8054629460698FAF7DFF805901C
S3150800792030490598FAF79DF80546FAF7F4FA81B250
S315080079302748C183C08B00902548838B0022542199
S31508007940FE2000F068FF2249088BFAF7A2FA2049C0
S315080079500190C88BFAF79DFA22490090FAF7BEF80B
S3150800796007460199FAF77DF806461A49FAF7B6F86E
S3150800797017490390088BFAF78CFA07461549FAF760
S31508007980ADF80646144801683046FAF766F80290DC
S315080079900399FAF7A3F805461149FAF709F8049086
S315080079A0FAF7B9FA84B20A48C08B0F49884204DB51
S315080079B00748C08B0D49884204DD0222FE21572064
S315080079C000F0C3FF05484038C485204607B0F0BD1F
S315080079D07802002000007A44900100200C04002060
S315080079E00000C84100247449B80B00008813000041
S315080079F0F0B587B000240020069005904049488BD2
S31508007A00FAF747FA07463F49FAF768F805463C4940
S31508007A10488BFAF73EFA3B490490FAF75FF80746AF
S31508007A20394801683846FAF718F806462946FAF733
S31508007A3055F806903549888BFAF72BFA06463449E5
S31508007A40FAF707F8054629460698FAF747F805901B
S31508007A5030490598FAF705F80546FAF75CFA81B24F
S31508007A6027488183C08B00902548838B00225421A8
S31508007A70FE2000F0D0FE2249488BFAF70AFA204980
S31508007A800190C88BFAF705FA22490090FAF726F80A
S31508007A9007460199F9F7E5FF06461A49FAF71EF867
S31508007AA017490390488BFAF7F4F907461549FAF788
S31508007AB015F80646144801683046F9F7CEFF0290D5
S31508007AC00399FAF70BF805461149F9F771FF04907F
S31508007AD0FAF721FA84B20D48403884850848808B25
S31508007AE00D49884204DB0648808B0C49884204DD30
S31508007AF00222FE21572000F028FF204607B0F0BDDD
S31508007B007802002000007A448C0100200C04002032
S31508007B100000C84100247449B80B0000881300000F
S31508007B20F0B587B000240020069005904049088BE0
S31508007B30FAF7AFF907463F49F9F7D0FF05463C493A
S31508007B40088BFAF7A6F93B490490F9F7C7FF0746E9
S31508007B50394801683846F9F780FF06462946F9F795
S31508007B60BDFF06903549088CFAF793F9064634495D
S31508007B70F9F76FFF054629460698F9F7AFFF05900E
S31508007B8030490598F9F76DFF0546FAF7C4F981B249
S31508007B9027484184408C00902548038C01225421B3
S31508007BA0FE2000F038FE2249088BFAF772F92049C0
S31508007BB00190488CFAF76DF922490090F9F78EFF83
S31508007BC007460199F9F74DFF06461A49F9F786FF60
S31508007BD017490390088BFAF75CF907461549F9F730
S31508007BE07DFF0646144801683046F9F736FF0290CD
S31508007BF00399F9F773FF05461149F9F7D9FE049079
S31508007C00FAF789F984B20A48408C0F49884204DB9E
S31508007C100748408C0D49884204DD0222FE21572080
S31508007C2000F093FE05484038C485204607B0F0BDED
S31508007C307802002000007A44900100200C040020FD
S31508007C400000C84100247449B80B000088130000DE
S31508007C50F0B587B000240020069005904049488B6F
S31508007C60FAF717F907463F49F9F738FF05463C4939
S31508007C70488BFAF70EF93B490490F9F72FFF0746A8
S31508007C80394801683846F9F7E8FE06462946F9F7FD
S31508007C9025FF06903549888BFAF7FBF806463449DE
S31508007CA0F9F7D7FE054629460698F9F717FF05900E
S31508007CB030490598F9F7D5FE0546FAF72CF981B249
S31508007CC027480184408C00902548038C01225421C2
S31508007CD0FE2000F0A0FD2249488BFAF7DAF8204981
S31508007CE00190088CFAF7D5F822490090F9F7F6FEC4
S31508007CF007460199F9F7B5FE06461A49F9F7EEFE61
S31508007D0017490390488BFAF7C4F807461549F9F757
S31508007D10E5FE0646144801683046F9F79EFE0290CD
S31508007D200399F9F7DBFE05461149F9F741FE049078
S31508007D30FAF7F1F884B20A48008C0F49884204DB46
S31508007D400748008C0D49884204DD0222FE2157208F
S31508007D5000F0FBFD054840388485204607B0F0BD95
S31508007D607802002000007A448C0100200C040020D0
S31508007D700000C84100247449B80B000088130000AD
S31508007D8070B5044600257E20FDF778F8A3480088DC
S31508007D9040280ADD0020A1490880A1490870FF2172
S31508007DA001319E48801DF9F7F8FD9D4800780300CB
S31508007DB0FDF7F5F8080521364760DAF1F0EF0020FF
S31508007DC0964948717E2C0FD1088001209449087085
S31508007DD0924801880088401C904A1080901D44549F
S31508007DE000201146C87002E000208C490880002057
S31508007DF08A4908710FE1FE2C01D0002C0FD1874863
S31508007E0001880088401C854A1080901D4454022031
S31508007E108349087010460079001911460871FAE07E
S31508007E207E4801880088401C7C4A1080901D445476
S31508007E3003207B490870104600790019114608711D
S31508007E40E9E0764801880088401C744A1080901D35
S31508007E5044540420724908701046007900191146E6
S31508007E6008710846C470C078002802D105206C49FC
S31508007E700870D0E069484079012856D15E2C1CD19B
S31508007E80664800797E30654908717E216348028814
S31508007E900088401C614B1880981D8154801FC0784B
S31508007EA0401EC0B21946C870002802DC05205C498D
S31508007EB0087000205949487155E05D2C1CD1574877
S31508007EC000797D30554908717D215448028800881B
S31508007ED0401C524B1880981D8154801FC078401E44
S31508007EE0C0B21946C870002802DC05204C49087043
S31508007EF000204A49487136E0484800790019474940
S31508007F000871084601880088401C444A1080901D64
S31508007F104454801FC078401EC0B21146C87000285D
S31508007F2021DC05203E4908701DE07D2C03D1012087
S31508007F303A49487117E039480079001937490871F4
S31508007F40084601880088401C344A1080901D445415
S31508007F50801FC078401EC0B21146C870002802DCD7
S31508007F6005202F49087056E02C480079C043401C6C
S31508007F70C5B27D2D05D15D2C17D10620284908707C
S31508007F8013E07E2D08D15E2C0FD1062024490870F7
S31508007F900BE03FE02FE011E0A54203D1062020497F
S31508007FA0087002E007201E4908701C4801880088EE
S31508007FB0401C1A4A1080901D44542CE0174801882A
S31508007FC00088401C154A1080901D44547E2C08D108
S31508007FD001211448017000201146088010490870D4
S31508007FE008E000200D49088000210E480170002095
S31508007FF00B4908700FE000200949087007480188F6
S315080080000088401C054A1080901D445400201146E3
S31508008010088000E000BF00BF70BD00009C0500207E
S31508008020F10100200C04002070B50246002013461A
S315080080300C461D02FF26360235402543284670BDEC
S3150800804086B004460D4626686768A0680590E0680D
S3150800805004902069039060690290A0690190E06924
S31508008060009017A0FCF75AFF31461BA0FCF756FFF5
S3150800807039461CA0FCF752FF1DA00599FCF74EFFD8
S315080080801EA00499FCF74AFF1FA00399FCF746FFB8
S3150800809020A00299FCF742FF23A00199FCF73EFFB6
S315080080A026A00099FCF73AFF2948416A29A0FCF75F
S315080080B035FF29462BA0FCF731FF00BFFEE700007D
S315080080C05B48617264206661756C742068616E64D1
S315080080D06C65725D0D0A00005230203D2025780D32
S315080080E00A0000005231203D2025780D0A000000C4
S315080080F05232203D2025780D0A0000005233203DDB
S315080081002025780D0A000000523132203D202578BE
S315080081100D0A0000537461636B6564204C52203D60
S315080081202025780D0A000000537461636B6564208E
S315080081305043203D2025780D0A00000053746163E2
S315080081406B656420505352203D2025780D0A0000A7
S3150800815000ED00E05343425F53484353523D2578B0
S315080081600D0A000043757272656E74204C52203DEC
S315080081702025780D0A000000064907488185002158
S315080081802C3041805F218180C1800181002141819D
S3150800819070470000FBAA00004C03002000B51549F3
S315080081A015488185FF210F312C3041800A21018134
S315080081B0A021C180C821818078214181B221C18155
S315080081C032210182BE2181810C4901830B4925395F
S315080081D04183052141820A218182C182084981831E
S315080081E0C183018441841221FDF79BFB02492C318E
S315080081F0888400BDFBAA00004C02002078210000FC
S315080082000410000010B57E20FCF738FEFEF762FE6B
S31508008210012800D110BD6048407801287ED15E480B
S315080082202030C07C002802D0012860D137E04021E8
S315080082305A48FAF7E7FE00281DD157482030807CB7
S31508008240012805D1002056494860534920318874D1
S315080082505348406D5349884220D2514840687D2191
S31508008260090188421AD24C4894384089002815D109
S31508008270FCF78CFB12E048482030807C002803D1AC
S3150800828001204549203188744548806E4549884211
S3150800829002D2FCF77BFB01E0FCF76AFC79E0404977
S315080082A04868FF21F531F9F735FBC007C00F0028EC
S315080082B00ED180210920C006FAF7AFFE0121374802
S315080082C0FAF7ABFE10210920C006FAF7A6FE0DE064
S315080082D080210920C006FAF79EFE10210920C00653
S315080082E0FAF799FE01212D48FAF795FE51E02A483A
S315080082F02030C07C052829D129494868FF21F53155
S31508008300F9F708FBC007C00F002810D18021092003
S31508008310C006FAF782FE0121204800E03AE0FAF7A3
S315080083207CFE10210920C006FAF777FE30E080218E
S315080083300920C006FAF76FFE10210920C006FAF7D1
S315080083406AFE01211548FAF766FE21E01248203038
S31508008350C07C06280ED180210920C006FAF75BFEEC
S3150800836010210920C006FAF756FE01210B48FAF734
S3150800837052FE0DE080210920C006FAF74EFE0121C3
S315080083800648FAF74AFE10210920C006FAF745FE04
S3150800839000BF00BF00BF3DE70C04002000040048F2
S315080083A00C02002030750000FBF7BCFDFBF710F946
S315080083B0FBF74EFAFAF736FBFAF7CEF80B20F9F781
S315080083C0FDFF0C20F9F7FAFF0920F9F7F7FF03205C
S315080083D0F9F7F4FF01219448FAF764F94B200002F3
S315080083E0FAF786FA0121914841700021C1700020F0
S315080083F08E4920310874C87301218C488171FBF7B6
S315080084001BF9FBF7C5FD1A216320FBF7EFFDFFF704
S31508008410C1F9FCF773F900F0A3F984489438408948
S31508008420002801D1FCF7B2FA7F217E20FCF764FD13
S3150800843000217E482038C17700207C492031087207
S31508008440F0E07A482038C07F0300FCF7A8FD08054D
S31508008450134D8B9EB1C4D7EAFAF74CF9FFF7D2FE53
S31508008460FDF77EFEFBF7E8F801F0D8FC7E20FCF766
S3150800847005FDD6E0002301221946184600F09AFCAD
S3150800848000231A461946184600F094FC68484068C6
S315080084906849884204D908216748FAF7BCFD1DE0F7
S315080084A063494868FF21F531F9F734FAC007C00F68
S315080084B000280ED180210920C006FAF7ACFD10214C
S315080084C00920C006FAF7A7FD01215B48FAF7A3FDC4
S315080084D004E010210920C006FAF79FFDFAF7B4F95F
S315080084E07E20FCF7CBFC9CE0FAF704F9FBF7A4F82E
S315080084F0002301221946184600F05CFC00231A46A0
S315080085001946184600F056FC4948406849498842C9
S3150800851004D908214848FAF77EFD1DE04449486811
S31508008520FF21F531F9F7F6F9C007C00F00280ED17B
S3150800853080210920C006FAF76EFD10210920C00621
S31508008540FAF769FD01213C48FAF765FD04E01021B8
S315080085500920C006FAF761FDFEF744FB7E20FCF70A
S315080085608DFC5EE0FDF7F0F920210920C006FAF738
S3150800857054FDFAF7BFF8FFF745FEFDF7F1FDFBF7E7
S315080085805BF87E20FCF77AFC4BE0FDF76FFB2021B9
S315080085900920C006FAF741FDFAF7ACF8FFF732FEF4
S315080085A0FDF7DEFDFBF748F87E20FCF767FC38E0B0
S315080085B0FDF7CAF920210920C006FAF72EFDFAF7B9
S315080085C099F8FFF71FFEFDF7CBFDFBF735F87E2080
S315080085D0FCF754FC25E0FDF749FB20210920C006DD
S315080085E0FAF71BFDFAF786F8FFF70CFEFDF7B8FD5C
S315080085F0FBF722F87E20FCF741FC12E0FDF7C4FCED
S3150800860020210920C006FAF708FDFAF773F8FFF7E4
S31508008610F9FDFDF7A5FDFBF70FF87E20FCF72EFC0C
S3150800862000BF00BF0DE70000002401400C04002035
S315080086300C020020204E000000040048FEB5464803
S315080086400088F9F726FC0746444881693846F9F751
S31508008650D9FC00D2FEBD414A11685068F9F7F9F90C
S315080086603E4988600A46D1689068F9F7F2F902909F
S315080086703A48C16801208007F9F7F3F900903748AE
S3150800868081680098F9F7E9F90746344801693846D8
S31508008690F9F78EF90446314948690299F9F7E1F97B
S315080086A001902E4A91695069F9F7DBF907462B487C
S315080086B0C1693846F9F712FA0546284881682846F6
S315080086C0F9F7CFF90546254A116A5069F9F7C9F944
S315080086D00746224881693846F9F700FA06462146D0
S315080086E03046F9F7BEF9064629460198F9F760F9C2
S315080086F007463146F9F75CF9184948622A20085EA8
S31508008700F9F7BCFB00901548416A0098F9F750F94B
S315080087100746F9F7E7FB00B2104948852A20085EA4
S31508008720898D884204DD0D48808D00B20B49488545
S315080087300A482A21415E002902DA002007494885AD
S315080087400648C0680549086108468068C860002070
S315080087500149088000BF7DE7500100204004002041
S3150800876010B540210F48F9F718F940210D48FAF7D6
S315080087703DFA06210B48FDF7D4F80A49898988424B
S315080087800AD108482C38808D0749884208D0FFF757
S31508008790F3FCFCF793FB03E0FFF7EEFCFCF78EFB1C
S315080087A010BD000078030020FBAA0000F7B5A0B0B2
S315080087B00C46154680216846F9F7EFF8002700268B
S315080087C07E2168460170FE214170EF2181700721E4
S315080087D0C170209901710021417184712112C17102
S315080087E001210172457229128172012605E0684647
S315080087F0805DC019C7B2701CC6B20B2EF7DBF843F2
S31508008800401CC1B26846C1727E2101730D21FBF777
S31508008810DFFF23B0F0BDFFB5A1B006461C462A9F70
S31508008820802101A8F9F7B9F80020009000257E21DB
S31508008830684601714671229981710721C171239990
S3150800884001720021417284722112C17201210173E1
S31508008850477339128173012507E001A8415D009825
S315080088600818C0B20090681CC5B20B2DF5DB00983D
S31508008870C043401CC1B26846C1737E2101740D21F4
S3150800888001A8FBF7A5FF25B0F0BDFFB585B00546E5
S315080088900E460E9F002001900290039004900090CF
S315080088A000247E2168460171457186710421C171D3
S315080088B0079901720899417287723912C1720124A7
S315080088C007E001A8015D00980818C0B20090601C76
S315080088D0C4B2082CF5DB0098C043401CC1B26846F8
S315080088E001737E2141730A2101A8FBF771FF09B0C4
S315080088F0F0BD7FB5044600200090019002900390D9
S31508008900002600257E2168460170FE2141708F21D0
S3150800891081700321C1700021017144712112817196
S31508008920012505E06846405D8019C6B2681CC5B2D7
S31508008930072DF7DBF043401CC1B26846C1717E21A2
S3150800894001720921FBF744FF7FBDF7B584B00546E0
S315080089500E46002000900190029003900027002404
S315080089607E2168460170467085700121C17069468E
S3150800897006980871012405E06846005DC019C7B26B
S31508008980601CC4B2052CF7DBF843401CC1B268462C
S3150800899041717E2181710721FBF71AFF07B0F0BDEF
S315080089A0F0B5ABB0074680210BA8F8F7F6FF002014
S315080089B0089009900A900590069007900026049062
S315080089C0DFA00490002400253B00FCF7E8FA060423
S315080089D04BC3F1EFEEEDFAF7DDFD044600200890F3
S315080089E009900A90E0B22104090E2202120E230E03
S315080089F0009201910290D4A2092108A8FCF79EFAD8
S31508008A007E2108A801730021417344218173132133
S31508008A10C1731522D1490CA8F8F7A6FF082208A9A0
S31508008A200EA80330F8F7A0FFC5A0049005220CA8ED
S31508008A3003300499F8F798FF012004E00BA9095CB4
S31508008A404919CDB2401C1728F8DBE843401CC1B2CF
S31508008A5010A8C17019267E21017119210BA8FBF7F0
S31508008A60B7FE69E1FAF796FD0446002008900990DA
S31508008A700A90E0B22104090E2202120E230E009279
S31508008A8001910290B0A2092108A8FCF757FAFAF753
S31508008A9087FD04460020059006900790E1B2200461
S31508008AA0000E2202120E230E009202910190A6A237
S31508008AB0092105A8FCF742FA7E2108A80173FE21C0
S31508008AC04173442181733321C1733622A4490CA80A
S31508008AD0F8F74AFF9AA0049005220CA803300499D7
S31508008AE0F8F742FF96A00490052212A80499F8F711
S31508008AF03BFF93A00490042213A803300499F8F7C7
S31508008B0033FF082208A90EA80330F8F72DFF042121
S31508008B1010A8C170082205A91330F8F725FF082206
S31508008B2008A916A80330F8F71FFF012004E00BA9CF
S31508008B30095C4919CDB2401C3728F8DBE843401CCC
S31508008B40C1B218A8C1707E21017139210BA8FBF7A3
S31508008B503FFEF1E07E2108A80173FE214173CF2173
S31508008B6081730621C1730021017475A00490052242
S31508008B700CA801300499F8F7F7FE012004E00BA9C8
S31508008B80095C4919CDB2401C0A28F8D3E843401CB1
S31508008B90052149000BAA50547E210B2011540C21A3
S31508008BA00BA8FBF715FEC7E0C5E057E02BE0FFE78B
S31508008BB07E2108A80173FE214173CE218173082105
S31508008BC0C1730021017467A0049007220CA8013024
S31508008BD00499F8F7C9FE012004E00BA9095C4919B4
S31508008BE0CDB2401C0C28F8D3E843401CC1B20C2077
S31508008BF00BAA11547E210D201154072041000BA801
S31508008C00FBF7E6FD98E07E2108A80173FE21417373
S31508008C10CD2181730821C1730021017451A00490EC
S31508008C2007220CA801300499F8F79EFE012004E0FB
S31508008C300BA9095C4919CDB2401C0C28F8D3E843A6
S31508008C40401CC1B20C200BAA11547E210D201154D0
S31508008C50072041000BA8FBF7BBFD6DE0FAF79AFC6D
S31508008C6004460020089009900A90E0B22104090EF3
S31508008C702202120E230E00920191029032A20921BD
S31508008C8008A8FCF75BF9FAF78BFC04460020059068
S31508008C9006900790E1B22004000E2202120E230E5F
S31508008CA000920291019028A2092105A8FCF746F92D
S31508008CB07E2108A80173FE214173CB21817300210F
S31508008CC00174012141741EA0049005220CA80330EA
S31508008CD00499F8F749FE0C260BA98819082205A954
S31508008CE0F8F742FE08360BA98819082208A9F8F7EA
S31508008CF03BFE0836701FC1B208A8C173C07B801E30
S31508008D00C1B208A88174012004E00BA9095C4919BD
S31508008D10CDB2401CB042F8DBE843401C0BA988558D
S31508008D20701CC6B27E208855701CC6B231460BA888
S31508008D30FBF74EFD00E000BF00BF2BB0F0BD000002
S31508008D405350726F42000000252E3258252E325895
S31508008D50252E3258252E325800000000A601002084
S31508008D60BB010020425F5631305F3400F8B5064635
S31508008D700C46F9F75FFA051E0F4600D0012001439D
S31508008D8049000B484908411AC90F0DD0002E01D0D9
S31508008D90012100E000210C4361004908401AC00F78
S31508008DA002D10120FCF756F928463946F8BD0000DD
S31508008DB00000F07F0FB591B0002010900F900E9034
S31508008DC00D900C90FE480078642803D0FD48C078C2
S31508008DD0642804D10121FB482038017103E00021F1
S31508008DE0F848203801711398002802D001287DD14F
S31508008DF073E21498002803D10021F2482038C17183
S31508008E00F148C1891298814203D1EF48C08A0F9070
S31508008E1001E005200F900F98052802DC05200F9029
S31508008E2004E00F98322801DB05200F900F9912985D
S31508008E30411A1198814222DDE2482038C07900287B
S31508008E4015D1E1486C384068DF496C39C861149817
S31508008E50012804D10121DB482038C17156E0149855
S31508008E60002853D10021D7482038C1714EE0149804
S31508008E7000284BD10021D3482038C17146E00F990C
S31508008E80129841181198814240DCCE482038C079A2
S31508008E9001283BD1CB484079012831D1CA486C38E2
S31508008EA04068C9496C39C969401AC84988420DD20F
S31508008EB0C448B4380089462822DDC248B438008937
S31508008EC0801E81B2BF48B438018119E0BE486C38AB
S31508008ED04068BD496C39C969401A7D2189018842B3
S31508008EE00ED9B848B43800895F2800E0FEE307DAEF
S31508008EF0B448B4380089801C81B2B248B4380181BC
S31508008F000121B048417100212038C171AD4820388F
S31508008F10C07901287ED1AB48C07C042803D0A94873
S31508008F20C07C052804D1002201210846FDF778FFF8
S31508008F300F991298411A119881426CDDA2486C3833
S31508008F4040687D21C900884207D264209C49087080
S31508008F5000219C4820388172B8E19A482038807AE6
S31508008F6000286DD10121974820388172964880895A
S31508008F7064285CDA93486038818DC08E081A81B2FD
S31508008F80904860380187008F0990F8F782FF0146FC
S31508008F900A908F480068F8F7A1FD0B90F8F7EEFFE6
S31508008FA08C4A03C287486038808F40430990F8F797
S31508008FB077FF0B910A9087480CC80A98F8F77EFE47
S31508008FC0844A03C2834903C9FFF7D0FE0B910A906E
S31508008FD0F8F7FCFF804908607A486038808F089067
S31508008FE0F8F757FF014609907B480068F8F776FDC1
S31508008FF07A490A90F8F735FD0B90F8F78CFF78490F
S3150800900008700846007864280DDC71480068F8F78F
S31508009010B5FF01E057E16CE00022724B0B910A9014
S31508009020F8F7C0FF06D864206D49087002E064208E
S315080090306B49087063486038818D4030418245E14C
S3150800904061486C38806C7D21C90088424CD9002063
S315080090505D496C3988646248007864283FDA594863
S315080090606038818D4030408A814233DD012189078D
S3150800907057480068F8F79CFC0B90F8F74CFF81B24C
S3150800908050486038828D4030408A101A814205DA8D
S3150800909053480078801E5249087020E049486038D5
S315080090A0818D4030408A081A0A90F8F7E7FE0B903F
S315080090B0474801680B98F8F7A5FF10D2484800788A
S315080090C0801C4749087008460078642807DD642034
S315080090D0087004E042480078401D41490870394844
S315080090E06038818D403041823D48007834490870A7
S315080090F0ECE034484079002876D1334880896428E2
S3150800910003DB64202E490870E0E02F486C3840687D
S315080091107D21C900884207D26420294908700021A8
S31508009120284820388172D1E026482038807A0028DD
S3150800913074D1012123482038817223488089642804
S3150800914063DA20486038818DC08E081A81B21D48BE
S3150800915060380187008F0990F8F79BFE01460A9050
S315080091601B480068F8F7BAFC0B90F8F707FF194A8E
S3150800917003C214486038808F40430990F8F790FE80
S315080091800B910A9013480CC80A98F8F797FD114AEC
S3150800919003C2104903C9FFF7E9FD0B910A90F8F7D6
S315080091A015FF0D49086007486038808F0890F8F762
S315080091B070FE0146099008480068F8F78FFC14E02D
S315080091C0F20000202C04002078020020701700000E
S315080091D0D4000020D8000020E00000200000C8428B
S315080091E0F10000200000F03F67E0FE490A90F8F71A
S315080091F038FC0B90F8F78FFEFB4908700846007894
S31508009200642805DD6420087002E06420F6490870C9
S31508009210F648818D4030418258E0FFE7F448806C7B
S315080092207D21C900884243D90020F1498864EF4866
S31508009230818D4030408A814231DD01218907ED4820
S315080092400068F8F7B5FB0B90F8F765FE81B2E748BA
S31508009250828D4030408A101A814205DAE248007849
S31508009260801EE14908701FE0E048818D4030408A41
S31508009270081A0A90F8F702FE0B90DE4801680B9868
S31508009280F8F7C0FE10D2D8480078801CD649087076
S3150800929008460078642807DD6420087004E0D24890
S315080092A00078401DD0490870D048818D40304182F1
S315080092B0CD480078D049087008E0CC485438007A80
S315080092C0CD49087002E00020CB490870CA480278E8
S315080092D014991398FDF7A4FD08E21498002803D101
S315080092E00021C24840300172C0486030C07C012865
S315080092F004D002287ED003287DD199E0BC486C3082
S3150800930041881298814204D1B9486C30408A0F903E
S3150800931001E00A200F90B64840687D21C9008842BE
S3150800932077D3B2484030407A002872D1AF48818F4F
S315080093304030018301214172008B0A90F8F7A9FD9C
S31508009340AE490B90F8F75EFE1AD8A8484030008B55
S315080093500790F8F79EFD01460890A948F8F7BEFB66
S31508009360A8490990F8F77DFBA7490A90F8F720FB6A
S315080093700B90F8F7D0FDC1B29C48603001713FE010
S315080093809A484030008BFF210A3188421ADC9748F8
S315080093904030008B0790F8F77CFD01460890974807
S315080093A0F8F79CFB97490990F8F75BFB96490A90F2
S315080093B0F8F7FEFA0B90F8F7AEFDC1B28B486030AD
S315080093C001711DE089484030008B0790F8F761FD70
S315080093D0014608908948F8F781FB8C490990F8F707
S315080093E040FB89490A90F8F7E3FA0B90F8F793FDE2
S315080093F0C1B202E00EE029E00BE07C486030017162
S315080094007A4860300079642803DB64217748603045
S31508009410017129E076486C3041881298814204D15E
S3150800942073486C30408A0F9001E00A200F901BE0C9
S315080094306F486C3081881298814204D16C486C3030
S31508009440808A0F9001E00A200F900DE068486C3082
S3150800945081881298814204D165486C30808A0F90C1
S3150800946001E00A200F9000BF00BF0F98052802DC14
S3150800947005200F9004E00F98322801DB32200F9068
S315080094805A4860308079002802D11198FDF76AFCA5
S315080094900F991298411A119881422ADB544840685C
S315080094A05349086200208863C86350491198488761
S315080094B008464030007A00280FD11498012807D1B1
S315080094C01E214A48603081700121203801720BE064
S315080094D0002146484030017206E01498002803D15E
S315080094E00021424840300172002140484030417115
S315080094F041E10F991298411811988142F8DC3B48CE
S315080095004030007A012809D10021384840300172DC
S315080095103748406836490862002088633348603017
S3150800952080790028E4D132486C30408A0A280BDB5F
S315080095302F48406A0A90F8F7ACFC35490B90F8F7C3
S31508009540CDFA3449086020E029486C30408A0A2858
S3150800955010DA27486C30408A07280BDD2448406A11
S315080095600A90F8F796FC2C490B90F8F7B7FA2949B0
S3150800957008600AE01E48406A0A90F8F78AFC2749FC
S315080095800B90F8F7ABFA2349086018484030808AF0
S315080095900890F8F77EFC0A9014484030808A0790B5
S315080095A0F8F777FC08901B4801680898F8F759FA05
S315080095B009900A99F8F755FA0B90F8F7DFFC184A5C
S315080095C003C20A4860300079401D0590F8F768FC28
S315080095D00991089005484030808A0190F8F774FC94
S315080095E005911FE00000C842F1000020CC030020CE
S315080095F00C020020D4000020F200002000007A436C
S31508009600000082430000BE42000040400000B44211
S3150800961000803B45CC0000200000FA440080BB4493
S31508009620E80000200490FB4903C9FFF79FFB03915C
S315080096300290059B049AF8F7A9FB07910690099BE7
S31508009640089AF8F73BFB0B910A90F8F779FC81B278
S31508009650F1488180FF386D38806A0A90F8F719FC5E
S31508009660EE490B90F8F73AFAED490860EA48943063
S31508009670C08A0890F8F70DFC0A90E7489430C08A2B
S315080096800790F8F706FC0890E54801680898F8F787
S31508009690E8F909900A99F8F7E4F90B90F8F76EFCDF
S315080096A0DC4A03C2DC48B4300079401D0590F8F75F
S315080096B0F7FB09910890D8489430C08A0190F8F7CA
S315080096C003FC05910490D34903C9FFF74FFB0391A7
S315080096D00290059B049AF8F759FB07910690099B97
S315080096E0089AF8F7EBFA0B910A9000E01BE2F8F7F4
S315080096F027FC81B2C848C180FF38013880896428B0
S3150800970027DAC84880890890F8F7C3FB0A90C54845
S315080097106C38406B0590F8F7BCFBC3490690F8F720
S31508009720DDF90890BF484188FF305530808E081A09
S315080097300690F8F7A3FB07900899F8F7CFF9099070
S315080097400A99F8F78EF9B9490B90F8F7C7F9B849A5
S315080097500860B1488088642802DB6421AE488180AD
S31508009760AD48C088642802DB6421AB48C18001216A
S31508009770A948B4308171A8489430007A00287AD074
S31508009780012879D1A448B4308078AA490978884252
S315080097900EDA0021A048B43081702038017200200A
S315080097A0A0496C39C86400219B48B430C17060E197
S315080097B00F991298411A119881420EDD96489430F5
S315080097C0407A012804D19448B4300179C17050E137
S315080097D064219148B430C1704BE18F48B430C07CE5
S315080097E00300FBF7DCFB06FD04098DFCFBFD8A483C
S315080097F0B4300179C1703BE18A486C38806B89497D
S315080098006C39C96B401A7D21C90088424DD98548F3
S315080098106C38806B83496C39C8637F485430418FF4
S31508009820119881420CDD7C4880880A3081B27A48DA
S315080098308180C088642834DB64217748C18030E0A1
S315080098400F980B9074485430418F1198411A0B9811
S31508009850C20F10184010401C81420EDA6E488088EC
S31508009860801C81B26C488180C088642819DB642119
S315080098706948C18015E0FDE03AE10F980B9066480B
S315080098805430418F1198411A0B98C20F1018401086
S31508009890801C814205DD60488088801E81B25E4852
S315080098A081805D495431119848875E486C38406814
S315080098B05C496C39096A401A5F49884211DD564885
S315080098C08088401D81B2544881808088642802DBE4
S315080098D064215148818053486C38406851496C3935
S315080098E008624D48B4308079002804D14A48B4301B
S315080098F00179C17003E048480179B430C170B7E016
S3150800990048486C38806B47496C39C96B401A7D21C9
S31508009910C90088424BD943486C38806B41496C3939
S31508009920C8633D485430418F119881420CDD3A484E
S31508009930C0880A3081B23848C180C088642832DBC2
S3150800994064213548C1802EE00F980B903248543078
S31508009950418F1198411A0B98C20F10184010401CDD
S3150800996081420CDA2C48C088801C81B22A48C18002
S31508009970C088642817DB64212748C18013E00F9844
S315080099800B9025485430418F1198411A0B98C20FF5
S3150800999010184010801C814205DD1F48C088801EB3
S315080099A081B21D48C1801C495431119848871D4809
S315080099B06C3840681B496C39096A401A1F49884245
S315080099C015DD1548C088401D81B21348C180C0887E
S315080099D0642802DB64211048C18002E034E00BE011
S315080099E042E010486C3840680E496C3908620A48EB
S315080099F08179B430C1703BE007489430C0790128BA
S31508009A001ED100200449B431C87000210248B43080
S31508009A10817018E0E8000020780300200000FA446E
S31508009A20CC0000207802002000007A440000C842DA
S31508009A30D4000020F200002088130000581B000004
S31508009A401E203B49C87000BF39482038C079012814
S31508009A5006D100213648C17000203549887002E0D9
S31508009A601E213348C17000BF32213148C17000BF82
S31508009A7000BF41E02E48C07C012829D10F991298D1
S31508009A804118119881421FDB2948B4380179B4304E
S31508009A90C1700F9912984018801E119988420FDDDF
S31508009AA024480078002822D12148B4388088401DEF
S31508009AB081B21F48B438818001201E49087016E01B
S31508009AC000201C49087012E000211948C1700EE0F8
S31508009AD01748C07C042803D01548C07C052803D144
S31508009AE000201349C87002E00A211148C17003E03A
S31508009AF000210F48C17000BF00BF0D48C07C012877
S31508009B0008D10B48C07802460B9014991398FDF7B4
S31508009B1087F907E00648807802460B90149913984F
S31508009B20FDF77EF900BF00BF109815B000BD000014
S31508009B302C040020F000002010B500220121084660
S31508009B40FDF76EF94C49888BF8F7A3F94B4908607D
S31508009B50FEF774FD48482030C07A002839D14848B5
S31508009B60464948604448808BB42807D04248808BD1
S31508009B70B32803D04048808BB52804D101203E493C
S31508009B802031487303E000203B49203148733D48A3
S31508009B90406E3D49884267D93748C08B801E3B498D
S31508009BA0098888420DDC3448C08B801C37490988EF
S31508009BB0884206DBFDF71CFF01202F492031C872B9
S31508009BC003E02D48C08B3149088000202D4948669E
S31508009BD04AE029482030C07A01283BD12C48274939
S31508009BE048602548808BE62809D02348808BFF21CA
S31508009BF02C31884203D02048808BE72804D10121E4
S31508009C001D482030417303E000201B49203148736A
S31508009C101C48406E1C49884226D91748C08B801EAE
S31508009C201A49098888420DDC1348C08B801C1749DD
S31508009C300988884206DBFEF70BF802200E49203118
S31508009C40C87203E00C48C08B1049088000200D49F3
S31508009C50486609E000200B494866084948850122FC
S31508009C60FE215720FEF771FE0448408DC2B201213D
S31508009C700020FDF7D5F810BD0C0400204004002094
S31508009C80000034430C020020881300000001002065
S31508009C900000664330B503465A480068181AFF2480
S31508009CA0F534A04201D957480360481E904248DD62
S31508009CB055480078002816D1881A3C2805DA881AEB
S31508009CC03C24201A514C207002E000204F4C207092
S31508009CD04E4800785524201A4C4C207020460078AF
S31508009CE04B4C20702AE04B480078002822D14A487D
S31508009CF00088401A07280ADD454C2078C40F241826
S31508009D006410424D2C7028460078414C2070424819
S31508009D100088401A012808DD3D480078401E3C4C62
S31508009D20207020460078394C20703B48028001207C
S31508009D30384C207036480078344C207036480280FB
S31508009D405DE0481E90424CDC481C824249DC2E48A5
S31508009D500078012828D12F48007800282AD12E48D3
S31508009D600088801A07280BDD294C2078C40F241890
S31508009D706410264D2C7028460078254C20700DE07E
S31508009D8025480088801A012808DB21480078401EEB
S31508009D901F4C2070204600781C4C20701E480280FC
S31508009DA001201C4C207005E017480078002801D1D6
S31508009DB0164C2070481E904205D115480078401E62
S31508009DC0124C20701BE08A4205D111480078001F0A
S31508009DD00E4C207013E00E480078801F0B4C207044
S31508009DE00DE00020094C20700A4C20700120064C1A
S31508009DF0207009480088824201DB07480280034830
S31508009E00007830BD04010020F8000020020100207F
S31508009E10030100200A0100200801002010B5FDF703
S31508009E2047FA01280AD1FD484068FF21F5318842E2
S31508009E3003D90421FA48F9F7EEF810BDF948407835
S31508009E4000287DD1F7492031487410210920C00621
S31508009E50F9F7E1F880210920C006F9F7DCF80121B5
S31508009E60EF48F9F7D8F80021EE482030C1740023EE
S31508009E70012219461846FEF79DFF00231A46194681
S31508009E801846FEF797FFE5484068FF21F5318842F6
S31508009E9009D2E4482030007C002803D10421E04898
S31508009EA0F9F7BBF8FCE20421DD48F9F7B4F800201D
S31508009EB0DC4920310874D9484068DB498842F1D921
S31508009EC0D8488079002823D120210920C006F9F72F
S31508009ED0A2F8D24840687D214901884201D2FAF7A2
S31508009EE019FD0821CE48F9F796F80021CD48C1702A
S31508009EF00020CC49203148710021CA4820308171A0
S31508009F000020C649486248637D20400148601DE03C
S31508009F10C4488078012819D10020C049486000212A
S31508009F20C048C1700020BF49203148710021BD4892
S31508009F30203081710020B94948624863B94900E078
S31508009F4017E02031C8740121B64841704021B44851
S31508009F50F9F758F80028A5D020210920C006F9F7F6
S31508009F605CF80021AF482030C174012120384170C7
S31508009F7096E2AC482030C07C0300FBF710F80705D2
S31508009F8089F9F7F6F5F488000021A6480172C1712F
S31508009F9001710020A1490864A24920314874087457
S31508009FA020210920C006F9F738F800219D482030FD
S31508009FB0417100209B49203188719849486248635D
S31508009FC00021984841720023012219461846FEF7D7
S31508009FD0F1FE00231A4619461846FEF7EBFE91488D
S31508009FE04038C18D8186C18D0186818D41868B4819
S31508009FF040687D21090188422BD900208B490870C9
S3150800A00040218748F8F7FEFF00281AD110210920B9
S3150800A010C006F9F700F880210920C006F8F7FBFF0B
S3150800A02001217F48F8F7F7FFFAF774FC08217C4806
S3150800A030F8F7F1FF7E20FAF721FF1E20F8F7B0FCAB
S3150800A04002E000207549486004217548F8F7E3FFE7
S3150800A0501DE040217248F8F7D5FF002804D10821F1
S3150800A0606F48F8F7DAFF03E008216D48F8F7D3FFE1
S3150800A0706A484068FF21F531884208D9694894380A
S3150800A0804089002803D104216548F8F7C4FF06E291
S3150800A09064484038818D418660484068FF21F53123
S3150800A0A0884204D204215E48F8F7B7FF03E004218A
S3150800A0B05B48F8F7B0FF594948687D21C900F7F7AA
S3150800A0C029FC23282ED2554948687D21C900F7F76F
S3150800A0D021FC192826D953484038818DFF38553830
S3150800A0E04088814207DA4F484038C18DFF385538D5
S3150800A0F0408881420DDB4B4820308079012821D1E8
S3150800A1000020464948600862022146482030C1744A
S3150800A11018E0002041494860086202204149203180
S3150800A120C8740FE03D4948687D21C900F7F7F2FB7E
S3150800A130232807D300203949486008620220394994
S3150800A1402031C874354A6C325188FF325532D08D69
S3150800A15001231A46FEF72EFE00231A46194618460C
S3150800A160FEF728FE9BE145E1D7E08CE03BE0FFE700
S3150800A1702C484038818D418628484068FF21F531B2
S3150800A180884204D204212648F8F747FF03E0042151
S3150800A1902348F8F740FF214841686C3000897D2242
S3150800A1A0D2005043814210D21C4A6C325188FF3289
S3150800A1B05532D08D01231A46FEF7FCFD00231A46B8
S3150800A1C019461846FEF7F6FD0CE0002115480172FF
S3150800A1D000201249486001211248417103201149A3
S3150800A1E02031C8745BE10F484038818D4186C08DA7
S3150800A1F0FF217D31884204DC0A484038808D884238
S3150800A20016DD0023012219461846FEF7D3FD002362
S3150800A2101A4619461846FEF7CDFD33E00C02002013
S3150800A220000400480C040020B80B0000C4000020FD
S3150800A2309E4948687D21C900F7F76CFB9B496C313C
S3150800A2404989884210D2994A6C329188FF32553230
S3150800A250D08D01231A46FEF7ADFD00231A4619468E
S3150800A2601846FEF7A7FD0DE09148818DC1860020AE
S3150800A2708E49486000218E484030017204208C497E
S3150800A2806031C8740BE18A48C08DFF217D31884250
S3150800A29003DC8748808D88420CDD0023012219469D
S3150800A2A01846FEF787FD00231A4619461846FEF794
S3150800A2B081FD31E07D4948687D21C900F7F72AFB11
S3150800A2C07A496C31098A0F3988421ED2774A6C322C
S3150800A2D0D189774A908D01230022FEF76BFD7448D9
S3150800A2E04030C079012806D10023012219461846B4
S3150800A2F0FEF760FD10E06D4A6C32D1886C4AD08D4D
S3150800A30001231A46FEF756FD06E000206749486015
S3150800A310052067496031C874C1E064484068FF2178
S3150800A320F531884204D204216248F8F776FE0FE038
S3150800A3305E484068FF21F531884209D95B48406884
S3150800A3404B21C900884203D204215A48F8F763FE14
S3150800A35056484068584988421ED2544A6C32D189B8
S3150800A360534A908D01230022FEF724FD50484030C1
S3150800A370C079012806D10023012219461846FEF79E
S3150800A38019FD36E0494A6C32D188494AD08D0123F5
S3150800A3901A46FEF70FFD2CE004214648F8F73DFE65
S3150800A3A0424840684449C831884222D300203F4980
S3150800A3B048603F486030C07B012804D106213C48EC
S3150800A3C06030C17405E0002139486030C174203816
S3150800A3D041700023012219461846FEF7EBFC0023BC
S3150800A3E01A4619461846FEF7E5FC04213148F8F7DF
S3150800A3F012FE54E000212E4840300172C1710171ED
S3150800A40000202A4908640865C86429496031087427
S3150800A41020210920C006F8F700FE002024496031F3
S3150800A42048718871214948624863002120484030B4
S3150800A43041720023012219461846FEF7BBFC002389
S3150800A4401A4619461846FEF7B5FC1948C18D818685
S3150800A450C18D0186818D41864030C07800281DD186
S3150800A460124840681549884218D9FAF753FA002065
S3150800A4700E4948600E4854384088032808DA0C48C4
S3150800A480C08D5A280ADC012109486030C17405E0EC
S3150800A490002107486030C1742038417000BF00BFF2
S3150800A4A07E20FAF7EBFC00BFC7E400000C02002090
S3150800A4B0CC03002000040048A438000060EA00002D
S3150800A4C0E0A40008C8000020440100006423000836
S3150800A4D030A500080C0200209C0800004450000823
S3150800A4E0015E2D01020304043506070809ACA24AD9
S3150800A4F0041A5916011129250A450181580B1058C5
S3150800A500594C4C3031313278010B11CB7E153E0453
S3150800A51001320505133812061459413230303532E6
S3150800A520384834353034324120041B7D5D7E0000C6
S705080018C515
